:020000040000FA
:10080000633A8DEF60F0FFFF6DEF04F00000000031
:100810000000000000000000186ED8CF19F0E0CFF3
:100820001AF00001E9CF20F0EACF1BF0E1CF1CF075
:10083000E2CF1DF0D9CF1EF0DACF1FF0F3CF27F0B3
:10084000F4CF28F0FACF29F0FBCF2AF000C022F035
:1008500001C023F002C024F003C025F004C026F03C
:100860009DAA36EF04F09EBAEBEF0FF09DA83CEF87
:1008700004F09EB809EF10F0A3AA42EF04F0A4BA66
:10088000B7EF0FF0A3A848EF04F0A4B8D5EF0FF02E
:1008900022C000F023C001F024C002F025C003F004
:1008A00026C004F020C0E9FF1BC0EAFF1B8E1CC05D
:1008B000E1FF1DC0E2FF1EC0D9FF1FC0DAFF27C045
:1008C000F3FF28C0F4FF29C0FAFF2AC0FBFF18502D
:1008D0001AC0E0FF19C0D8FF10002D6ED8CF2EF03F
:1008E000E0CF2FF00001E9CF35F0EACF30F0E1CFD3
:1008F00031F0E2CF32F0D9CF33F0DACF34F0F3CFAA
:100900003CF0F4CF3DF0FACF3EF0FBCF3FF000C01B
:1009100037F001C038F002C039F003C03AF004C02B
:100920003BF09DA097EF04F09EB016EF0FF0A0A251
:100930009DEF04F0A1B2A2EF0FF037C000F038C075
:1009400001F039C002F03AC003F03BC004F035C0FA
:10095000E9FF30C0EAFF308E31C0E1FF32C0E2FF74
:1009600033C0D9FF34C0DAFF3CC0F3FF3DC0F4FF11
:100970003EC0FAFF3FC0FBFF2D502FC0E0FF2EC04E
:10098000D8FF1000F2CF21F0F29CF29EA60FF66E77
:10099000090EF722000EF86E0900F55021BCF28C0A
:1009A00021BEF28E120000000000000000000000D6
:1009B000000084008A00A4001900120001009100C8
:1009C0009700B4001E0015000102AB00B200D50074
:1009D00028001C000106C500CD00F50032002300F0
:1009E0000200D800E1000D013C002A000204E800EA
:1009F000F2002101460031000206F6000101330138
:100A00004B0035000300FF000A013D015000380093
:100A100003020F011B0152015A003F00030620018F
:100A20002D0167016400460004002E013B0179019D
:100A30006E004D0004023C014A018A017800540016
:100A400004064301510192017D00580005004A014E
:100A500058019B0182005B00050258016701AD014E
:100A60008C006200050666017501BE0196006900F2
:100A7000060072018201CD01A000700006027D0116
:100A80008D01DB01AA007600060683019301E201D5
:100A9000AF007900070089019901EA01B4007B00E9
:100AA00007029501A701F901BE0081000706A10117
:100AB000B3010802C80087000800AC01BE0115029E
:100AC000D2008C000802B601C9012202DC009200AB
:100AD0000806BB01CE012802E10095000900C00113
:100AE000D3012F02E60098000902CB01DF013B028F
:100AF000F0009E000906D501E9014802FA00A300B2
:100B00000A00DF01F30154020401A9000A02E8010E
:100B1000FC0160020E01AF000A06ED01020266024E
:100B20001301B1000B00F20107026C021801B400BE
:100B30000B02FA01110277022201BA000B0604022D
:100B4000190283022C01C0000C000C0222028D024B
:100B50003601C5000C0215022B0298024001CB00A1
:100B60000C0419022F029D024501CE000C051E0245
:100B70003502A2024A01D1000C0626023D02AD0256
:100B80005401D8000C082F024702B8025E01DE00B3
:100B90000D0037025002C3026801E5000D02400259
:100BA0005902CD027201EB000D0444025D02D20233
:100BB0007701EE000D0548026102D8027C01F100C8
:100BC0000D0650026A02E2028601F8000D08590281
:100BD0007302ED029001FE000E0060027A02F6023E
:100BE0009A0104010E0267028202FF02A4010B01B6
:100BF0000E046B0285020303A9010E010E056F02AC
:100C00008A020803AE0111010E0676029202110358
:100C1000B80118010E087E0299021B03C2011E01D1
:100C20000F008502A0022303CC0124010F028B02D6
:100C3000A7022C03D6012B010F048F02AB02300355
:100C4000DB012E010F059302AF023503E0013101F4
:100C50000F069A02B6023E03EA0134010F08A10210
:100C6000BE024703F40137011000A802C502500379
:100C7000FE013B011002AF02CC02580308023E0104
:100C80001004B302D0025C030D023F011005B6024E
:100C9000D3026103120241011006BD02DB026903A7
:100CA0001C0244011008C402E2027203260247013A
:100CB0001100CA02E802790330024B011102D0028E
:100CC000EE0281033A024E011104D302F2028503BF
:100CD0003F024F011105D602F5028903440251017A
:100CE0001106DD02FC0291034E0254011108E302D9
:100CF00003039903580257011200E9020A03A103F2
:100D000062025A011202F0021003A8036C025E0193
:100D10001204F3021203AC0371025F011205F50223
:100D20001603B003760261011206FC021D03B8032C
:100D300080026401120803032403C0038A026701CE
:100D4000130009032A03C80394026A0113020F0364
:100D50003003D0039E026E01130412033403D30345
:100D6000A3026F01130515033703D703A80271010E
:100D700013061C033D03DF03B202740113082103B1
:100D80004403E603BC0277011400FF03FF03FF03E3
:100D9000C6027A011400F2CF21F0F29CF29EF76AAB
:100DA000BA0FF66E0D0EF722000EF86E0900F55020
:100DB00021BCF28C21BEF28E1200BA08DD07780841
:100DC0007908F609F709080A0000F2CF21F0F29C31
:100DD000F29EF76AEE0FF66E0D0EF722000EF86E19
:100DE0000900F55021BCF28C21BEF28E12000000E9
:100DF000080100007EFF3CC300000000000100006D
:100E00000000007E00C300200042800000247E24F9
:100E100060005A42784264423C423E4270007E4248
:100E20007C4200000000000C1042003050825E1234
:100E3000764278831E0078811E4216423E02664248
:100E400018816A00064C0E00661466187E00564231
:100E50007E08564A381210816E0006246628003C2F
:100E60006C42182400000018000000280800F2CF8F
:100E700021F0F29CF29EF76A920FF66E0E0EF722A8
:100E8000000EF86E0900F55021BCF28C21BEF28EE6
:100E900012002020312E38204D485A00F2CF21F088
:100EA000F29CF29EF76AC00FF66E0E0EF722000E4D
:100EB000F86E0900F55021BCF28C21BEF28E1200B2
:100EC0002020332E35204D485A00F2CF21F0F29CDD
:100ED000F29EF76AEE0FF66E0E0EF722000EF86E17
:100EE0000900F55021BCF28C21BEF28E12002020A8
:100EF000352E33204D485A00F2CF21F0F29CF29E5D
:100F0000F76A1C0FF66E0F0EF722000EF86E09003E
:100F1000F55021BCF28C21BEF28E12002020372E1B
:100F200030204D485A00F2CF21F0F29CF29EF76A31
:100F30004A0FF66E0F0EF722000EF86E0900F550FC
:100F400021BCF28C21BEF28E12002031302E3120D5
:100F50004D485A00F2CF21F0F29CF29EF76A780FCA
:100F6000F66E0F0EF722000EF86E0900F55021BC48
:100F7000F28C21BEF28E12002031342E30204D48EA
:100F80005A00F2CF21F0F29CF29EF76AA60FF66E9D
:100F90000F0EF722000EF86E0900F55021BCF28CFE
:100FA00021BEF28E12002031382E31204D485A00D9
:100FB000F2CF21F0F29CF29EF76AD40FF66E0F0E7C
:100FC000F722000EF86E0900F55021BCF28C21BE0C
:100FD000F28E12002032312E30204D485A00F2CFCE
:100FE00021F0F29CF29EF76A020FF66E100EF722C5
:100FF000000EF86E0900F55021BCF28C21BEF28E75
:1010000012002032342E39204D485A00F2CF21F000
:10101000F29CF29EF76A300FF66E100EF722000E69
:10102000F86E0900F55021BCF28C21BEF28E120040
:101030002032382E30204D485A00F2CF21F0F29C59
:10104000F29EF76A5E0FF66E100EF722000EF86E33
:101050000900F55021BCF28C21BEF28E1200203521
:10106000302E30204D485A00F2CF21F0F29CF29EF3
:10107000F76A8C0FF66E100EF722000EF86E09005C
:10108000F55021BCF28C21BEF28E120020494E5642
:10109000414C49440000F2CF21F0F29CF29EF76AE5
:1010A000BA0FF66E100EF722000EF86E0900F5501A
:1010B00021BCF28C21BEF28E12004B4559205445C2
:1010C00053540000F2CF21F0F29CF29EF76AE80F31
:1010D000F66E100EF722000EF86E0900F55021BCD6
:1010E000F28C21BEF28E12004C45442054455354DC
:1010F0000000F2CF21F0F29CF29EF76A160FF66E16
:10110000110EF722000EF86E0900F55021BCF28C8A
:1011100021BEF28E120020485600F2CF21F0F29C40
:10112000F29EF76A3E0FF66E110EF722000EF86E71
:101130000900F55021BCF28C21BEF28E1200205421
:101140004D50202020430000F2CF21F0F29CF29E6F
:10115000F76A6C0FF66E110EF722000EF86E09009A
:10116000F55021BCF28C21BEF28E12002043555264
:101170000000F2CF21F0F29CF29EF76A960FF66E15
:10118000110EF722000EF86E0900F55021BCF28C0A
:1011900021BEF28E1200205057520000F2CF21F0F3
:1011A000F29CF29EF76AC00FF66E110EF722000E47
:1011B000F86E0900F55021BCF28C21BEF28E1200AF
:1011C000205357520000F2CF21F0F29CF29EF76AB2
:1011D000EA0FF66E110EF722000EF86E0900F550B8
:1011E00021BCF28C21BEF28E120020444953000033
:1011F000F2CF21F0F29CF29EF76A140FF66E120EF7
:10120000F722000EF86E0900F55021BCF28C21BEC9
:10121000F28E1200504B484F4C4420310000F2CF68
:1012200021F0F29CF29EF76A420FF66E120EF72240
:10123000000EF86E0900F55021BCF28C21BEF28E32
:101240001200504B484F4C4420300000F2CF21F0A8
:10125000F29CF29EF76A700FF66E120EF722000EE5
:10126000F86E0900F55021BCF28C21BEF28E1200FE
:101270005041524D205253540000F2CF21F0F29CC5
:10128000F29EF76A9E0FF66E120EF722000EF86EAF
:101290000900F55021BCF28C21BEF28E12005041A3
:1012A000524D204C4400F2CF21F0F29CF29EF76A9E
:1012B000CA0FF66E120EF722000EF86E0900F550F6
:1012C00021BCF28C21BEF28E1200202044454D4FED
:1012D00020200000F2CF21F0F29CF29EF76AF80F76
:1012E000F66E120EF722000EF86E0900F55021BCC2
:1012F000F28C21BEF28E1200204B5041353030204E
:101300000000F2CF21F0F29CF29EF76A260FF66EF3
:10131000130EF722000EF86E0900F55021BCF28C76
:1013200021BEF28E120020202020204441590000CE
:10133000F2CF21F0F29CF29EF76A540FF66E130E74
:10134000F722000EF86E0900F55021BCF28C21BE88
:10135000F28E120020202020204F46460000F2CFBF
:1013600021F0F29CF29EF76A820FF66E130EF722BE
:10137000000EF86E0900F55021BCF28C21BEF28EF1
:10138000120020203438303020420000F2CF21F00B
:10139000F29CF29EF76AB00FF66E130EF722000E63
:1013A000F86E0900F55021BCF28C21BEF28E1200BD
:1013B00020203936303020420000F2CF21F0F29C5C
:1013C000F29EF76ADE0FF66E130EF722000EF86E2D
:1013D0000900F55021BCF28C21BEF28E12002031A2
:1013E0003932303020420000F2CF21F0F29CF29EE0
:1013F000F76A0C0FF66E140EF722000EF86E090055
:10140000F55021BCF28C21BEF28E1200203338340C
:10141000303020420000F2CF21F0F29CF29EF76AB9
:101420003A0FF66E140EF722000EF86E0900F55012
:1014300021BCF28C21BEF28E120020202020202020
:101440004B330000F2CF21F0F29CF29EF76A680F56
:10145000F66E140EF722000EF86E0900F55021BC4E
:10146000F28C21BEF28E1200202020202042434424
:101470000000F2CF21F0F29CF29EF76A960FF66E12
:10148000140EF722000EF86E0900F55021BCF28C04
:1014900021BEF28E12002020414E414C4F470000E9
:1014A000F2CF21F0F29CF29EF76AC40FF66E140E92
:1014B000F722000EF86E0900F55021BCF28C21BE17
:1014C000F28E1200202053455249414C0000F2CFC9
:1014D00021F0F29CF29EF76AF20FF66E140EF722DC
:1014E000000EF86E0900F55021BCF28C21BEF28E80
:1014F000120020202020204E4F520000F2CF21F079
:10150000F29CF29EF76A200FF66E150EF722000E7F
:10151000F86E0900F55021BCF28C21BEF28E12004B
:101520002020202020204F4E0000F2CF21F0F29CFE
:10153000F29EF76A4E0FF66E150EF722000EF86E49
:101540000900F55021BCF28C21BEF28E1200202041
:101550002020535442590000F2CF21F0F29CF29E19
:10156000F76A7C0FF66E150EF722000EF86E090072
:10157000F55021BCF28C21BEF28E120020202020DA
:101580004F5045520000F2CF21F0F29CF29EF76AD4
:10159000AA0FF66E150EF722000EF86E0900F55030
:1015A00021BCF28C21BEF28E1200204449534142EC
:1015B0004C450000F2CF21F0F29CF29EF76AD80F62
:1015C000F66E150EF722000EF86E0900F55021BCDC
:1015D000F28C21BEF28E12002020454E41424C4535
:1015E0000000F2CF21F0F29CF29EF76A060FF66E31
:1015F000160EF722000EF86E0900F55021BCF28C91
:1016000021BEF28E120020202020204E2F4100000B
:10161000F2CF21F0F29CF29EF76A340FF66E160EAE
:10162000F722000EF86E0900F55021BCF28C21BEA5
:10163000F28E12001700414C432054485220000003
:1016400018004154544E2052454C00001A004241AB
:101650004E44204348470000100044454D4F202091
:10166000202000000F0046414E2043544C20000033
:101670000200465720524556202000001E00494EC9
:1016800048494220494E000005014C434420414452
:101690004A20000006014C434420425254200000DE
:1016A00007014C4544204252542000000800505786
:1016B000522041444A2000001D005057522D4F4EE9
:1016C000202000000D00524144494F2020200000FE
:1016D0000B00525332333220502000000A00525384
:1016E00032333220582000001B00534552204E5503
:1016F0004D2000001C0053455220504F4C4C000020
:101700001500535045414B45522000000E005452E5
:101710002054696D65200000F2CF21F0F29CF29E0A
:10172000F76A3C0FF66E170EF722000EF86E0900EE
:10173000F55021BCF28C21BEF28E120048492043A4
:10174000555252200000F2CF21F0F29CF29EF76A2F
:101750006A0FF66E170EF722000EF86E0900F550AC
:1017600021BCF28C21BEF28E120043555252204908
:1017700032200000F2CF21F0F29CF29EF76A980F1F
:10178000F66E170EF722000EF86E0900F55021BC18
:10179000F28C21BEF28E120048492054454D502053
:1017A0000000F2CF21F0F29CF29EF76AC60FF66EAF
:1017B000170EF722000EF86E0900F55021BCF28CCE
:1017C00021BEF28E1200505752494E204849000067
:1017D000F2CF21F0F29CF29EF76AF40FF66E170E2C
:1017E000F722000EF86E0900F55021BCF28C21BEE4
:1017F000F28E1200434E5452204552520000F2CF56
:1018000021F0F29CF29EF76A220FF66E180EF72274
:10181000000EF86E0900F55021BCF28C21BEF28E4C
:10182000120036305620484947480000F2CF21F0D8
:10183000F29CF29EF76A500FF66E180EF722000E19
:10184000F86E0900F55021BCF28C21BEF28E120018
:101850005245464C204849200000F2CF21F0F29C2E
:10186000F29EF76A7E0FF66E180EF722000EF86EE3
:101870000900F55021BCF28C21BEF28E12004B45BE
:10188000592048454C440000F2CF21F0F29CF29ED2
:10189000F76AAC0FF66E180EF722000EF86E09000C
:1018A000F55021BCF28C21BEF28E12005041204432
:1018B000495353200000F2CF21F0F29CF29EF76AC8
:1018C000DA0FF66E180EF722000EF86E0900F550CA
:1018D00021BCF28C21BEF28E1200504F555420488C
:1018E00049200000F2CF21F0F29CF29EF76A080F27
:1018F000F66E190EF722000EF86E0900F55021BCA5
:10190000F28C21BEF28E12004741494E20455252C0
:101910000000F2CF21F0F29CF29EF76A360FF66ECD
:10192000190EF722000EF86E0900F55021BCF28C5A
:1019300021BEF28E1200363056204661696C0000DE
:10194000F2CF21F0F29CF29EF76A640FF66E190E48
:10195000F722000EF86E0900F55021BCF28C21BE72
:10196000F28E120032373056204552520000F2CF2C
:1019700021F0F29CF29EF76A920FF66E190EF72292
:10198000000EF86E0900F55021BCF28C21BEF28EDB
:1019900012004641554C542020200000F2CF21F087
:1019A000F29CF29EF76AC00FF66E190EF722000E37
:1019B000F86E0900F55021BCF28C21BEF28E1200A7
:1019C00041544E20544553540000F2CF21F0F29C74
:1019D000F29EF76AEE0FF66E190EF722000EF86E01
:1019E0000900F55021BCF28C21BEF28E12005E542B
:1019F00053543100F2CF21F0F29CF29EF76A180F97
:101A0000F66E1A0EF722000EF86E0900F55021BC92
:101A1000F28C21BEF28E120049463B46413B4642C3
:101A20003B005350000A23E0010A4DE0030A5AE04C
:101A3000010AD8B464D0070AD8B46CD0010AD8B46B
:101A400074D0030AD8B47CD0010AD8B484D00F0A69
:101A5000D8B48CD0010AD8B494D0030AD8B4A0D09A
:101A6000010AD8B4B0D0070AD8B4BFD0D0D06651DC
:101A7000655D28E041AA26D0495224E1036A6651F7
:101A8000550FE96E000E0320EA6EEFCF54F0036AA3
:101A90006651550FE96E000E0320EA6EFF0EEF6EE1
:101AA000662B0F0E66170701586B576B54507F0853
:101AB00003E3010E536E05D05450FE0802E10C0EF4
:101AC000536E0001A7D0838E0701572BD8B4582B33
:101AD000585303E157514F0803E2586B576B532A91
:101AE000000198D0839E0701572BD8B4582B585328
:101AF00003E15751040801E2532A00018BD054AC92
:101B000002D0000E01D0010EE8A0839EE8B0838EC3
:101B1000532A80D054AA02D0000E01D0010EE8A0B2
:101B2000839EE8B0838E532A75D054A802D0000E4D
:101B300001D0010EE8A0839EE8B0838E532A6AD0BC
:101B400054A602D0000E01D0010EE8A0839EE8B09A
:101B5000838E532A5FD054A402D0000E01D0010E10
:101B6000E8A0839EE8B0838E532A54D054A202D0BA
:101B7000000E01D0010EE8A0839EE8B0838E532AA8
:101B800049D054A002D0000E01D0010EE8A0839EDF
:101B9000E8B0838E0701586B576B532A00013AD087
:101BA000839E0701572BD8B4582B5851000809E2DF
:101BB000FF0A03E15751F30804E20B0E536E586B12
:101BC000576B000127D0839E0701572BD8B4582BA1
:101BD0005851000808E2FF0A03E15751F30803E2F5
:101BE000536A586B576B000115D0839E0701572B22
:101BF000D8B4582B58510A0808E2FF0A03E157519C
:101C0000B70803E2536A586B576B000103D0839EF9
:101C1000536A00D037EF0FF0875317E1010E6525A7
:101C20000F0B665D0FE0036A6551550FE96E000EFC
:101C30000320EA6E61C9EFFF652B0F0E6517010ED9
:101C4000016E06D0020E016E03D0536A000E016EC3
:101C5000000CFF6BFE6B01011C6B056B046B1F6BB3
:101C60000001000C8A9A8A986A9D6A8F4192F1DF7E
:101C7000000C875326E141AA24D009015F6B5F5114
:101C80000F081BE3036A5F51550FE96E000E032036
:101C9000EA6EEF503F0B606F6051340803E0605113
:101CA000330809E1036A5F51550FE96E000E032006
:101CB000EA6EFF0EEF6E5F2BE2D7330E616F00010D
:101CC000ABDFD0DF000C09015E935E9141B25E8113
:101CD00007014C5303E04C2F01D0418409015E936E
:101CE00041BE5E8344AE03D05E9384AA5E83000E41
:101CF00084B8010E5F6F000E42B2010E5F11606F7B
:101D0000000E44BA010E6011616F000E5EB3010E49
:101D10006111FF0A4198E8B0418842A406D05E9163
:101D2000495203E10001A5DF0901495000010AE021
:101D3000010A1FE0030A36E0010A54E0070AD8B49A
:101D40006BD030D009015EA113D000016F5170112A
:101D5000D8B402D009010CD041B802D0090108D092
:101D60008B924194020E07014C6F010E496E0901DE
:101D70005AD06F51701104E109015EB105D0000124
:101D80008B82496A0CD0090141A409D0419441A831
:101D900004D0918C020E496E02D08B82496A0901EF
:101DA00042D000016F51701104E109015EB109D008
:101DB0000001919C040E07014C6F4194496E10D0B4
:101DC000090141B80ED0419442A205D0010E07018D
:101DD0004C6F04D00901BEC04CF70701030E496ED9
:101DE000090121D06F51701106E141B404D00901FD
:101DF0005EB109D00001919C040E07014C6F419423
:101E0000496E08D0090141A806D007014C6B4194E6
:101E1000020E496E090107D041A403D041948B8280
:101E2000496A090100D000019FEF0FF0CD90680EC4
:101E3000CE2409015A6FF00ECF205B6F5BC9CFFF34
:101E40005AC9CEFFCD809E900701487148A10BD0A2
:101E5000D6500101396FD7CF3AF1D76AD66A070158
:101E6000489384B848830001875301E1DAD507011C
:101E700048A163D048B347D048B545D001013A5393
:101E800006E13951C708D8A002D007013CD03A5129
:101E900007014B5D14E305E10101395107014A5D7A
:101EA0000EE30101395107014A5D09015C6F01012F
:101EB0003A5107014B5909015D6F0CD007014A5196
:101EC0000101395D09015C6F07014B5101013A596C
:101ED00009015D6F5D5310E15C5103080DE30701DB
:101EE000492B4951010806E23AC138F139C137F1AD
:101EF000020E496F03D009010701496B3AC14BF744
:101F000039C14AF701D0496B489548B348854180AB
:101F10004D2AD8B44E2A4E5000080FE2FF0A03E1C2
:101F20004D50F3080AE2010E4F26D8B0502AD8B41B
:101F3000512AD8B4522A4E6A4D6A0001C4D69E90E6
:101F40009DEF04F0B1908451B22409015A6F000151
:101F50008551B32009015B6F5BC9B3FF5AC9B2FF5A
:101F6000B180A1928A76A19200019DEF04F0A3AA0C
:101F700019D0A4AA17D06ECF56F9010E07013F253C
:101F8000405D0AE03F513F2B1C0FE96E050EEA6EE3
:101F9000D8B0EA2A56C9EFFFA4AA02D00001EBD7B5
:101FA000A49A0001A49A48EF04F007013D513E5D58
:101FB0000AE03D513D2B1C0FE96E040EEA6ED8B0CD
:101FC000EA2AEFCF6DFF3D513E5D01E1A398A49851
:101FD000000148EF04F09DAA19D09EAA17D0AECFF9
:101FE00056F9010E040119251A5D0AE01951192B41
:101FF000940FE96E020EEA6ED8B0EA2A56C9EFFFD6
:102000009EAA02D00001EBD79E9A00019E9A48EF4B
:1020100004F004011751185D0AE0940E1725E96ECB
:10202000010EEA6ED8B0EA2AEFCFADFF172B175199
:10203000185D01E19D989E98000148EF04F0090E9B
:10204000EA6E280EE96EEF500EE0050E016E006A92
:10205000002EFED7012EFBD72E0E006E002EFED7CF
:1020600000D0EF2EF2D7000CC00E8A6EFF0E8B6EE2
:10207000200E8C6E800E8D6EFF0E8E6EE60E8F6EB5
:10208000F00E906EB30E916EFF0E926EC00E936EB8
:10209000D00E946E600E956E7F0E966E976EE60E65
:1020A000986E300E996E010E9A6EF18E416A426AF8
:1020B000020E09012B6FC69A2B2D03D0300EC66E6F
:1020C00002D0320EC66EC76AC68A0D0E006E002E92
:1020D000FED79182918E8A90850ECD6EF00ECF6ED6
:1020E000680ECE6EA10ED56E000E0509CA6E680E82
:1020F000CB6E850EB16E85C0B3FF84C0B2FF8B94EA
:102100000C0EBD6E796AB66A230EBE6EBD50CF0B43
:10211000BD6E849E9198919E020E006E002EFED799
:102120000000316BC9CF32F931C9C9FFC7A0FED752
:10213000C9CF32F9326B3251010802E3322BFBD79F
:10214000080E316FC9CF32F931C9C9FFC7A0FED718
:10215000C9CF32F9326B3251010802E3322BFBD77F
:10216000010E316FC9CF32F931C9C9FFC7A0FED7FF
:10217000C9CF32F9326B3251010802E3322BFBD75F
:10218000316BC9CF32F931C9C9FFC7A0FED7C9CF5A
:1021900032F9326B3251010802E3322BFBD7020EC7
:1021A000006E002EFED70000918E9188010E2B6FDD
:1021B000C69A2B2D03D0300EC66E02D0320EC66EDC
:1021C000C76AC68A0D0E006E002EFED70F0E286F4E
:1021D000000135DF9D80C00EF212E4EF63F04196FE
:1021E0000101366B4A6AC150C00B0109C16EC05073
:1021F000C00B0409C06EC08EC2800901226B22513F
:102200000D0815E3D8902235036AFA0FE96E000E27
:102210000320EA6EEC6AED52EF6A036A22511A0F4C
:10222000E96E010E0320EA6EEF6A222BE8D7000167
:10223000AD6BAC6BADC0ABF0ACC0AAF0AF6BAE6B2E
:10224000B16BB06BB36BB26BB56BB46BB76BB66B9A
:10225000D96BD86B0101356B346B35C133F134C1A7
:1022600032F133C131F132C130F131C12FF130C11E
:102270002EF1366B3E6B3D6B406B3F6B426B416B9F
:10228000446B436B466B456B4A6B496B3B6B000180
:10229000756B746B776B766B796B786B7B6B7A6B2A
:1022A0007D6B7C6B7F6B7E6B816B806BE6EF63F08D
:1022B000F2CF41F9F29CF29E3EC9AAFF3DC9A9FFA7
:1022C000A69CA69EA680A850090141BDF28C41BFE4
:1022D000F28E406F403D2ED03EC949F93DC948F9C4
:1022E0003FC94AF949C9AAFF48C9A9FF4AC9A8FF75
:1022F000A69CA69EA684F2CF4BF9F29CF29E550EA8
:10230000A76EAA0EA76EA6824B51F212A6B2FED7F6
:10231000A692F2CF41F9F29CF29E3EC9AAFF3DC9B6
:10232000A9FFA69CA69EA680A85041BDF28C41BFE5
:10233000F28E406F40C901F00001000C9188090144
:102340003E6B070E3D6F0A0E3F6F0001B1DF01507B
:102350000F0B866F000C09013D513F03F3CF01F0D5
:10236000F4CF00F04003F35000263E513F03F350FA
:102370000020026E0001000C09013E51036E3D5128
:102380003D2BD8B43E2B416F03C042F93F51436F00
:10239000446B42C949F941C948F943C94AF949C995
:1023A000AAFF48C9A9FF4AC9A8FFA69CA69EA68461
:1023B000F2CF4BF9F29CF29E550EA76EAA0EA76EB5
:1023C000A6824B51F212A6B2FED7A6923E51036EE0
:1023D0003D513D2BD8B43E2B416F03C042F940C95B
:1023E00043F9446B42C949F941C948F943C94AF91B
:1023F00049C9AAFF48C9A9FF4AC9A8FFA69CA69E29
:10240000A684F2CF4BF9F29CF29E550EA76EAA0E4F
:10241000A76EA6824B51F212A6B2FED7A692000179
:10242000000CF2CF42F9F29CF29E3FC9AAFF3EC9CE
:10243000A9FFA69CA69EA680A850090142BDF28CC9
:1024400042BFF28E416F4151405D1DE03FC949F9E5
:102450003EC948F940C94AF949C9AAFF48C9A9FF74
:102460004AC9A8FFA69CA69EA684F2CF4BF9F29C6F
:10247000F29E550EA76EAA0EA76EA6824B51F212BF
:10248000A6B2FED7A6920001000C09013E6BFE0E1B
:102490003D6F3F6B00010CDF01C03AF909013E6B53
:1024A0003AC93DF9406B060E3F6F000154DF01C091
:1024B0003BF90901010E02243C6F0F0E3717010E84
:1024C00000018625006E003AF00E0016005009014A
:1024D00037133C51036E3B513B2BD8B43C2B3D6F23
:1024E00003C03EF94F503F6F406B416B426B3EC99A
:1024F00049F93DC948F93FC94AF949C9AAFF48C93C
:10250000A9FF4AC9A8FFA69CA69EA684F2CF4BF9B4
:10251000F29CF29E550EA76EAA0EA76EA6824B5194
:10252000F212A6B2FED7A6923C51036E3B513B2B52
:10253000D8B43C2B3D6F03C03EF950C040F951C0A8
:1025400041F952C042F9436B4051446F456B466BB1
:10255000476B3EC949F93DC948F944C94AF949C9D7
:10256000AAFF48C9A9FF4AC9A8FFA69CA69EA6849F
:10257000F2CF4BF9F29CF29E550EA76EAA0EA76EF3
:10258000A6824B51F212A6B2FED7A6923C51036E20
:102590003B513B2BD8B43C2B3D6F03C03EF951C09F
:1025A00040F952C041F9426B436B4051446F456B57
:1025B000466B476B3EC949F93DC948F944C94AF9D8
:1025C00049C9AAFF48C9A9FF4AC9A8FFA69CA69E57
:1025D000A684F2CF4BF9F29CF29E550EA76EAA0E7E
:1025E000A76EA6824B51F212A6B2FED7A6923C511C
:1025F000036E3B513B2BD8B43C2B3D6F03C03EF9DF
:102600003EC949F93DC948F937C94AF949C9AAFF3C
:1026100048C9A9FF4AC9A8FFA69CA69EA684F2CFD6
:102620004BF9F29CF29E550EA76EAA0EA76EA682DB
:102630004B51F212A6B2FED7A6923CC93EF93BC955
:102640003DF939C940F938C93FF9000195DE090162
:102650003A2B3A9F3F6BFE0E3E6F3AC940F900019C
:10266000E0DE000CF2CF3DF9F29CF29E38C9AAFFE1
:1026700037C9A9FFA69CA69EA680A85009013DBD0A
:10268000F28C3DBFF28E396F010E37253D6F000E83
:1026900038213E6FF2CF3FF9F29CF29E3EC9AAFF6D
:1026A0003DC9A9FFA69CA69EA680A8503FBDF28C5E
:1026B0003FBFF28E3A6F3AC93CF939C93BF93BC981
:1026C00001F03CC902F00001000CF2CF29F9F29CA4
:1026D000F29EAA6AFD0EA96EA69CA69EA680A85090
:1026E000090129BDF28C29BFF28E246F243D01D04F
:1026F00008D0010E376F396B24C938F90001C5DEE7
:1027000009013F6BFD0E3E6F406B00018ADE09013F
:102710003E6BFE0E3D6F3F6B0001CADD01C022F92A
:10272000010E0901225D7F0B236F3E6B23C93DF92A
:10273000406B060E3F6F00010EDE0901010E022400
:102740002A6F030E0124256F000E2A21266F2651C1
:10275000036E2551252BD8B4262B296F03C02AF9E7
:10276000F2CF2BF9F29CF29E2AC9AAFF29C9A9FF30
:10277000A69CA69EA680A8502BBDF28C2BBFF28EE5
:10278000246F24510F0B1CE126C938F925C937F9EC
:10279000000168DF02C028F901C027F9010E090114
:1027A0002725296F000E28212A6F26C93EF925C941
:1027B0003DF9406F29C93FF90001DEDDB5D00901BF
:1027C0003E6B22C93DF9406B060E3F6F0001C3DD31
:1027D00001C025F90901010E0224266F2651036E5E
:1027E0002551252BD8B4262B296F03C02AF92AC9D5
:1027F00049F929C948F94A6B49C9AAFF48C9A9FF3B
:102800004AC9A8FFA69CA69EA684F2CF4BF9F29CCB
:10281000F29E550EA76EAA0EA76EA6824B51F2121B
:10282000A6B2FED7A6922651036E2551252BD8B409
:10283000262B296F03C02AF92AC949F929C948F961
:102840004A6B49C9AAFF48C9A9FF4AC9A8FFA69C63
:10285000A69EA684F2CF4BF9F29CF29E550EA76E6F
:10286000AA0EA76EA6824B51F212A6B2FED7A6926E
:102870002651036E2551252BD8B4262B296F03C072
:102880002AF92AC949F929C948F94A6B49C9AAFF4D
:1028900048C9A9FF4AC9A8FFA69CA69EA684F2CF54
:1028A0004BF9F29CF29E550EA76EAA0EA76EA68259
:1028B0004B51F212A6B2FED7A6922651036E2551B5
:1028C000252BD8B4262B296F03C02AF92AC949F928
:1028D00029C948F94A6B49C9AAFF48C9A9FF4AC989
:1028E000A8FFA69CA69EA684F2CF4BF9F29CF29E6E
:1028F000550EA76EAA0EA76EA6824B51F212A6B273
:10290000FED7A69226C93EF925C93DF9406B3F6B1B
:10291000000132DD0901222B229F3F6BFE0E3E6F2C
:1029200022C940F900017DDDF5EF63F009013A6B42
:1029300037513A5D1DE236C903F03551352BD8B415
:10294000362B3B6F03C03CF9036A3A513825E96ED8
:1029500039510320EA6EEFCF3DF93CC93FF93BC93D
:102960003EF93DC940F900015CDD09013A2BE0D791
:102970000001F9EF14F00901346B2F51345D20E2AE
:10298000036A34513025E96E31510320EA6E345127
:102990002D25376F000E2E21386FF2CF39F9F29CBA
:1029A000F29E38C9AAFF37C9A9FFA69CA69EA68099
:1029B000A85039BDF28C39BFF28EEF6E342BDDD7C3
:1029C00030C9E9FF31C9EAFFEF3C01D006D030C978
:1029D000E9FF31C9EAFFEF5231E12EC936F92DC9BD
:1029E00035F92FC937F933C939F932C938F9000136
:1029F0009DD70901346B2F51345D20E2036A3451B5
:102A00003025E96E31510320EA6E34512D25376FA0
:102A1000000E2E21386FF2CF39F9F29CF29E38C9A0
:102A2000AAFF37C9A9FFA69CA69EA680A85039BDBB
:102A3000F28C39BFF28EEF6E342BDDD7000187EFB9
:102A400018F0016A026A006A036A0901535102E13F
:102A5000525118E0100E546FD8905037513700364D
:102A600003365351035C02E15251005C07E35251BB
:102A7000005ED8A003065351035ED88001360236AB
:102A8000542FEAD70001000C09014F814D5304E097
:102A90004B2B4D514B5D4D6F036A4B514925E96EF0
:102AA0004A510320EA6EEF6A4B533FE0200E4E6F0F
:102AB0004751481104E14FB102D04C530DE048C9D1
:102AC00051F947C950F9536B0A0E526F0001B9DF33
:102AD0000901300E00244E6F4B07036A4B51492504
:102AE000E96E4A510320EA6E4EC9EFFF4D530DE0E7
:102AF0004B514D5D0AE14B07036A4B514925E96E85
:102B00004A510320EA6E2E0EEF6E48C951F947C9AB
:102B100050F9536B0A0E526F000193DF02C048F95F
:102B200001C047F909014F91BFD7010E016E0001A5
:102B3000000C036A4B5009014E25516F4F51032081
:102B4000526F50512E0811E14B520EE04B500808C5
:102B50000BE35151D8B45207510751C9E9FF52C98B
:102B6000EAFFEF504009EF6E24D04B50070821E3F5
:102B70005051270808E151C9E9FF52C9EAFFEF5057
:102B80008009EF6E16D050515F0802E2200E505FB0
:102B9000200E505F51C9E9FF52C9EAFFEF50C00B48
:102BA000EF6E51C9E9FF52C9EAFFEF505011EF6EC5
:102BB0004B2A0001000C44C94BF00901466B4551FA
:102BC000465D14E2036A46514225E96E43510320F3
:102BD000EA6EEFCF47F941C94FF940C94EF947C9ED
:102BE00050F90001A6DF0901462BE9D70001000CCE
:102BF0000901416B8A0E406F3DC943F93CC942F956
:102C00003EC944F93FC945F90001D5DF000C33C97D
:102C100048F932C947F9090E09014A6F360E496F62
:102C200035C94BF94C6B4D6B00012EDF090E0901C4
:102C30003D6F360E3C6F34C93EF935C93FF900018E
:102C4000D7DF000C09012D51010A000111E0030A30
:102C500013E0010A1EE0070A27E0010A48E0030A20
:102C600068E0010AD8B471D0070AD8B48CD08BD0F0
:102C70001E0E0701A56F89D009013E6B040E3D6F42
:102C80001E0E3F6F000158EC11F001C0A5F70701BF
:102C90007CD009013F6B040E3E6FA5C740F90001CF
:102CA00011EC12F0070171D00701A55163081EE372
:102CB000010EA527D890A53509012E6F2F6B2F3750
:102CC000C80E2E25306F000E2F21316F3133303377
:102CD00031333033313330C9B8FF31333131300B18
:102CE000006EB750CF0B0010B76E07014ED0070132
:102CF000A55302E0010EA55FD890A53509012E6FFE
:102D00002F6B2F37C80E2E25306F000E2F21316FFD
:102D10003133303331333033313330C9B8FF3133AD
:102D20003131300B006EB750CF0B0010B76E07017A
:102D30002CD00901336BA5C732F9050E346F030E91
:102D4000356F000164DF070120D0D8900701A53559
:102D500009012E6F2F6B2F37C80E2E25306F000EF6
:102D60002F21316F3133303331333033313330C988
:102D7000B8FF31333131300B006EB750CF0B00103C
:102D8000B76E070102D0070100D0A55164081EE20A
:102D90001E0EA56FD890A53509012E6F2F6B2F370A
:102DA000C80E2E25306F000E2F21316F3133303396
:102DB00031333033313330C9B8FF31333131300B37
:102DC000006EB750CF0B0010B76E0701A5C701F01A
:102DD0000001000C09014F6B8A0E4E6F32C950F989
:102DE0000001A7DE000C09012D51010A00010FE0CE
:102DF000030A11E0010A1CE0070A25E0010A2AE0A3
:102E0000030A2FE0010A4DE0070A56E055D0060EEE
:102E10000701A66F53D009013E6B050E3D6F060EEC
:102E20003F6F000158EC11F001C0A6F7070146D032
:102E300009013F6B050E3E6FA6C740F9000111EC7A
:102E400012F007013BD00701A651070802E3010E6B
:102E5000A62734D00701A651010802E2010EA65FA1
:102E60002DD00701A62D11D009012E6B2E51000186
:102E700081EC09F0000908E009012E2B326F0001F6
:102E8000A9DF0901F3D700010AD00901336BA6C7F6
:102E900032F9060E346F020E356F0001B8DE0701FD
:102EA0000DD0010E0701A65D0E0DF3CF2EF909011D
:102EB0002EC974FF070102D0070100D0A6510808EF
:102EC00002E2060EA66FA6C701F00001000C090180
:102ED0002D51010A00010FE0030A11E0010A1BE075
:102EE000070A24E0010A29E0030A2EE0010A38E07B
:102EF000070A42E041D0060E0701A76F3FD0090143
:102F00003E6B060E3D6F3F6F000158EC11F001C0A3
:102F1000A7F7070133D009013F6B060E3E6FA7C725
:102F200040F9000111EC12F0070128D00701A75168
:102F3000070802E3010EA72721D00701A7510108C6
:102F400002E2010EA75F1AD00901336BA7C732F95D
:102F5000060E346F020E356F000159DE07010ED0E8
:102F6000080ED8800701A7550E0DF3CF2EF90901E1
:102F70002EC971FF070102D0070100D0A751080830
:102F800002E2060EA76FA7C701F00001000C0901BD
:102F90003451070802E2070E346F3351070802E28A
:102FA000070E336F33C94BF04B50345D0AE3036AAD
:102FB0004B503125E96E32510320EA6EEF6A4B2AFD
:102FC000F3D74B6A0001000C91926AC031F9C9CF66
:102FD00032F931C9C9FFC7A0FED7C9CF32F90901FB
:102FE000326B3251010802E3322BFBD769C031F951
:102FF000C9CF32F931C9C9FFC7A0FED7C9CF32F94D
:10300000326B3251010802E3322BFBD768C031F931
:10301000C9CF32F931C9C9FFC7A0FED7C9CF32F92C
:10302000326B3251010802E3322BFBD767C031F912
:10303000C9CF32F931C9C9FFC7A0FED7C9CF32F90C
:10304000326B3251010802E3322BFBD7918200012F
:10305000000C0901326B8A0E316F336B070E346F2F
:10306000000195DF6A6B6AC069F069C068F068C0EA
:1030700067F0AADF4B6A8F900C0EB76E696A6A6AB6
:103080008F96736E8F98706E070E09012D6F000179
:10309000D9DD070E09012D6F0001A5DE070E09011C
:1030A0002D6F000114DF000C200E0901246F4B0E60
:1030B000256F500E266F410E276F350E286F300E8C
:1030C000296F2A6F200E2B6F2C6B090E236F240E95
:1030D000226F456A4B6A3E6B0A0E3D6F3F6B0001E3
:1030E00058EC11F001C088F088510508D8A0886B11
:1030F00009012E6B500E2D6F080E2F6F316B9A0E3B
:10310000306F23C933F922C932F9000134D4010EDA
:10311000A56F770EA46F100E896F020E09012D6F37
:10312000000190DD020E09012D6F00015CDE020E30
:1031300009012D6F0001CBDE8CDFF7EF63F0090191
:103140002651070B006E2631016E013201321F0E2F
:10315000011601502825E96E000E2921EA6E016A48
:10316000012A002A01D00136002EFDD7275303E0A3
:103170000150EF1203D0011E0150EF160001000CA8
:1031800009012335006E0036FC0E0016C250C30B39
:103190000010C26E420E006E002EFED70000000E20
:1031A00084B8010E23C926F9276F010E296F2A0E54
:1031B000286F0001C4DFC282C2B2FED7C4CF25F996
:1031C0000901C3CF24F9000E84B8010E23C926F9E2
:1031D000276F010E296F2C0E286F0001B0DF090147
:1031E0002551030823E303E12451EF081FE3D8909E
:1031F0002335036ADA0FE96E000E0320EA6E25C953
:10320000ECFFED5224C9EFFFD8902335036AFA0F83
:10321000E96E000E0320EA6E2451EF24016E255161
:10322000EC20ED5201C0EFFFEC6E01D08382036A07
:1032300023511A0FE96E010E0320EA6EEF2A0001F6
:10324000000C0901246B236B245324E123517F08D4
:1032500021E324C949F923C948F9FF0E4A6F49C936
:10326000AAFF48C9A9FF4AC9A8FFA69CA69EA68492
:10327000F2CF4BF9F29CF29E550EA76EAA0EA76EE6
:10328000A6824B51F212A6B2FED7A692232BD8B437
:10329000242BDAD70001B9EF19F009012A51010AEC
:1032A000000111E0030A11E0010A10E0040A0FE036
:1032B000030A0EE0010A10E0030A12E00E0A34E0ED
:1032C000080A39E038D0449A37D036D035D034D0D7
:1032D00044BA01D0448A30D044AA01D0449A2CD0B8
:1032E00044BA11D009012C6B2C51000198EC09F063
:1032F000000908E009012C2B326F00016BDD090188
:10330000F3D7000110D009012C6B2C5100017EEC89
:103310000AF0000908E009012C2B326F00015ADD88
:103320000901F3D7000108D009012B5302E1449AA7
:1033300001D0448A000100D044AA02D0010E01D07D
:10334000000E016E000C0B0E0901236F000118DF47
:10335000F131036EF031026E0332023202C022F903
:1033600009012251C00808E22251D90805E30001F1
:1033700068D70D0E896F09012251DA0809E2080E9B
:103380002A6F010E2B6F000188DF0F0E896F090174
:103390000001F9EF63F009012751010A00010FE074
:1033A000030A10E0010A1AE0070A23E0010A28E0F4
:1033B000030A2CE0010A4BE0070A4BE04AD0070160
:1033C000A86B49D009013E6B010E3D6F3F6B0001B8
:1033D00058EC11F001C0A8F707013DD009013F6B7F
:1033E000010E3E6FA8C740F9000111EC12F0070171
:1033F00032D00701A851F90802E3010EA8272BD00B
:103400000701A85302E0010EA85F25D00701A853C9
:1034100011E10901286B2851000198EC09F000091D
:1034200008E00901282B326F0001D4DC0901F3D731
:1034300000010BD00901336BA8C732F9050E346FB8
:10344000030E356F000107EC16F0070104D00701E9
:1034500002D0070100D0A851FA0801E2A86BA8C762
:1034600001F00001000C09012A51010A00011AE0D3
:10347000030A22E0010A64E0070AD8B49AD0010ADC
:10348000D8B4ACD0030AD8B4BDD0010AD8B4CFD0D8
:103490000F0AD8B4CDD0010AD8B4DAD0090AD8B40A
:1034A000F4D0F3D0036A8651C00FE96E000E0320FA
:1034B000EA6E140EEF6EEAD009012B3D22D02C6B80
:1034C0002C510B081DE3036A2C51C00F016E000E36
:1034D000032201C02DF903C02EF9200E2C252F6FD9
:1034E0003E6B3D6F140E3F6F000158EC11F02EC97A
:1034F000EAFF2DC9E9FF01C0EFFF09012C2BE0D73E
:103500001DD0036A00018651C00F016E000E032218
:1035100001C02DF903C02EF9200E000186250901F6
:103520002F6F3E6B3D6F140E3F6F000158EC11F092
:103530002EC9EAFF2DC9E9FF01C0EFFF0001A6D0A7
:1035400009012B3D1CD02C6B2C510B0817E3200ECE
:103550002C252D6F036A2C51C00FE96E000E03203D
:10356000EA6EEFCF2EF93F6B2DC93EF92EC940F917
:10357000000111EC12F009012C2BE6D718D0200E17
:103580000001862509012D6F036A00018651C00FD5
:10359000E96E000E0320EA6EEFCF2EF909013F6BB2
:1035A0002DC93EF92EC940F9000111EC12F00001BD
:1035B0006DD0036A8651C00FE96E000E0320EA6EDB
:1035C000EF5027080AE3036A8651C00FE96E000E28
:1035D0000320EA6E010EEF24EF6E58D0036A865185
:1035E000C00FE96E000E0320EA6EEF520AE0036A94
:1035F0008651C00FE96E000E0320EA6E010EEF5CEB
:10360000EF6E44D0036A8651C00FE96E000E0320AE
:10361000EA6E500EEF2409012E6F336B326F050EE8
:10362000346F030E356F000107EC16F02FD02ED04B
:1036300009012B5128080AE3036A00018651C00FD3
:10364000E96E000E0320EA6E2BC9EFFF00011ED0C9
:10365000036A8651C00FE96E000E0320EA6EEF5038
:10366000280809E2036A8651C00FE96E000E0320A4
:10367000EA6E140EEF6E036A8651C00FE96E000EFB
:103680000320EA6EEFCF01F027D000D0036A865105
:10369000C00FE96E000E0320EA6EEF50280809E221
:1036A000036A8651C00FE96E000E0320EA6E140E05
:1036B000EF6E036A8651C00FE96E000E0320EA6EBA
:1036C000EFCF2CF90901036A2C51A90FE96E070EFF
:1036D0000320EA6EEFCF01F00001000C09012A512E
:1036E000010A00010FE0030A10E0010A1AE0070ACC
:1036F00022E0010A26E0030A2AE0010A5DE0070A47
:103700005CE05BD04C0EBF6F59D009013E6B0B0ED5
:103710003D6F4C0E3F6F000158EC11F001C0BFF03F
:103720004DD009013F6B0B0E3E6FBFC040F9000149
:1037300011EC12F043D0BF51510802E3060EBF272F
:103740003DD0BF51280802E2060EBF5F37D0090105
:103750003E6BBFC03DF9406B0C0E3F6F0001ABEC00
:1037600011F002C02CF901C02BF9060E0901012449
:10377000016E000E0220036E0150F2CF2DF9F29C73
:10378000F29E03C0F7FF0001C2EC04F00900F5CF80
:1037900003F009012DBDF28C2DBFF28E2E6F03C0F8
:1037A0002FF903C033F9326F050E346F030E356FF6
:1037B000000107EC16F002D001D000D0BF5127085D
:1037C00003E2BF51520802E24C0EBF6FBFC001F0CE
:1037D000000C9D9A9D9809012C51FC0F25E2040FC5
:1037E000000118EF1CF07E86400EAF6E030E7F6E58
:1037F000A60EAC6E090118D07E86A00EAF6E010E2B
:103800007F6EA60EAC6E09010FD07E960C0EAF6EC9
:10381000A20EAC6E090108D07E96190EAF6EA60EF0
:10382000AC6E090101D009019D8A9D880001000C40
:10383000F2CF21F0F29CF29EE824F76AF736610F8E
:10384000F66E380EF722000EF86EFB6E0A00F55089
:10385000FA6E0800F55021BCF28C21BEF28EF96E92
:10386000E637F8370A38183809012A51010A0001E9
:1038700014E0030A15E0010A1FE0070A28E0010A24
:103880002DE0030A31E0010AD8B480D00F0AD8B481
:1038900082D0080AD8B48BD08AD00701D26B89D0E5
:1038A00009013E6B0C0E3D6F3F6B000158EC11F0AF
:1038B00001C0D2F707017DD009013F6B0C0E3E6FAE
:1038C000D2C740F9000111EC12F0070172D00701D4
:1038D000D251020802E3010ED2276BD00701D25366
:1038E00002E0010ED25F65D00701D251FC0F4DE21C
:1038F000040F0001E1EF1CF009012C6B2C510001B9
:10390000AFEC09F0000908E009012C2B326F00012F
:10391000EAEC16F00901F2D7070137D009012C6B48
:103920002C510001C6EC09F0000908E009012C2B1C
:10393000326F0001EAEC16F00901F2D7070125D039
:1039400009012C6B2C510001DDEC09F0000908E0A5
:1039500009012C2B326F0001EAEC16F00901F2D7B5
:10396000070113D009012C6B2C510001F4EC09F074
:10397000000908E009012C2B326F0001EAEC16F077
:103980000901F2D7070101D0070113D0D2C72CF9E2
:1039900020DF07010ED009012B51030806E32BC9D4
:1039A000D2F7D2C72CF9000114DF070102D00701BA
:1039B00000D0D251030801E2D26BD2C701F000015E
:1039C000000CF2CF21F0F29CF29EE824F76AF73661
:1039D000F30FF66E390EF722000EF86EFB6E0A003A
:1039E000F550FA6E0800F55021BCF28C21BEF28E23
:1039F000F96EF8381C3940396439A39AA398090143
:103A00002C51FC0F25E2040F00012CEF1DF07C86E9
:103A1000400E6F6E030E7D6EA60E6C6E090118D0FF
:103A20007C86A00E6F6E010E7D6EA60E6C6E090177
:103A30000FD07C960C0E6F6EA20E6C6E090108D032
:103A40007C96190E6F6EA60E6C6E090101D00901ED
:103A5000A38AA3880001000CF2CF21F0F29CF29E11
:103A6000E824F76AF736890FF66E3A0EF722000E51
:103A7000F86EFB6E0A00F550FA6E0800F55021BC96
:103A8000F28C21BEF28EF96E0E3A203A323A403A6A
:103A900009012A51010A000114E0030A16E0010A93
:103AA00021E0070A2AE0010A2FE0030A33E0010AB5
:103AB000D8B482D00F0AD8B484D0080AD8B48DD034
:103AC0008CD0030E0701D36F8AD009013E6B0D0E17
:103AD0003D6F030E3F6F000158EC11F001C0D3F7AA
:103AE00007017DD009013F6B0D0E3E6FD3C740F932
:103AF000000111EC12F0070172D00701D351020846
:103B000002E3010ED3276BD00701D35302E0010E6D
:103B1000D35F65D00701D351FC0F4DE2040F0001C4
:103B2000F8EF1DF009012C6B2C510001AFEC09F0EE
:103B3000000908E009012C2B326F0001EAEC16F0B5
:103B40000901F2D7070137D009012C6B2C51000174
:103B5000C6EC09F0000908E009012C2B326F0001C6
:103B6000EAEC16F00901F2D7070125D009012C6B08
:103B70002C510001DDEC09F0000908E009012C2BB3
:103B8000326F0001EAEC16F00901F2D7070113D0F9
:103B900009012C6B2C510001F4EC09F0000908E03C
:103BA00009012C2B326F0001EAEC16F00901F2D763
:103BB000070101D0070113D0D3C72CF91EDF07017D
:103BC0000ED009012B51030806E32BC9D3F7D3C745
:103BD0002CF9000112DF070102D0070100D0D351F8
:103BE000030802E2030ED36FD3C701F00001000CFB
:103BF000F2CF21F0F29CF29EE824F76AF736210F0B
:103C0000F66E3C0EF722000EF86EFB6E0A00F550C1
:103C1000FA6E0800F55021BCF28C21BEF28EF96ECE
:103C2000243B483B6C3B903B09012D51010A0001AC
:103C300014E0030A14E0010A1DE0070A25E0010A66
:103C400029E0030A2CE0010AD8B478D00F0AD8B4CE
:103C500076D0080AD8B47BD07AD0876B79D00901A6
:103C60003E6B0E0E3D6F3F6B000158EC11F001C032
:103C700087F06ED009013F6B0E0E3E6F87C040F992
:103C8000000111EC12F064D08751020802E3010E2A
:103C900087275ED0875302E0010E875F59D0875196
:103CA000FC0F4BE2040FAFEF1EF009012F6B2F51F9
:103CB00000010BEC0AF0000909E009012F2B326F1B
:103CC0000001EAEC16F00901F2D7000136D0090133
:103CD0002F6B2F51000122EC0AF0000909E00901C5
:103CE0002F2B326F0001EAEC16F00901F2D7000128
:103CF00024D009012F6B2F51000139EC0AF0000983
:103D000009E009012F2B326F0001EAEC16F00901DE
:103D1000F2D7000112D009012F6B2F51000150EC96
:103D20000AF0000909E009012F2B326F0001EAECCB
:103D300016F00901F2D7000100D00AD009D009011C
:103D40002E51030802E32EC987F0000101D000D0F4
:103D50008751030801E2876B87C001F0000CF2CFA6
:103D600021F0F29CF29EE824F76AF7368F0FF66E88
:103D70003D0EF722000EF86EFB6E0A00F550FA6E4B
:103D80000800F55021BCF28C21BEF28EF96EAA3CDF
:103D9000CE3CF23C163D09012A51010A000111E016
:103DA000030A12E0010A1BE0070A23E0010A28E0E7
:103DB000030A2CE0010A37E00F0A3CE0080A41E060
:103DC00040D00701D46B3FD009013E6B3D6B3F6B88
:103DD000000158EC11F001C0D4F7070134D00901FB
:103DE0003F6B3E6BD4C740F9000111EC12F00701A4
:103DF0002AD00701D451310802E3010ED42723D081
:103E00000701D45302E0010ED45F1DD00901336BCA
:103E1000D4C732F9060E346F020E356F000107EC7D
:103E200016F0070110D0010E0701D4250001BE6F66
:103E3000070109D00701D451320802E32BC9D4F796
:103E400002D0070100D0D451320801E2D46BD4C7AC
:103E500001F00001000C09012A51010A000111E0E2
:103E6000030A12E0010A1CE0070A25E0010A2CE01F
:103E7000030A32E00E0A52E00F0A5AE0070A5AE03B
:103E800059D00701D56B58D009013E6B100E3D6F1C
:103E90003F6B000158EC11F001C0D5F707014CD081
:103EA00009013F6B100E3E6FD5C740F9000111ECC0
:103EB00012F0070141D00701D551050802E3010EB8
:103EC000D527D5C74AF038D00701D55302E0010EF7
:103ED000D55FD5C74AF030D00701D55312E10901AB
:103EE0002C6B2C51000167EC0AF0000909E0090174
:103EF0002C2B326F0001EAEC16F00901F2D7000119
:103F00000BD00901336BD5C732F9070E346F010EA0
:103F1000356F000107EC16F007010ED009012B5197
:103F2000060802E32BC9D5F7D5C74AF0070104D02C
:103F3000070102D0070100D0D551060801E2D56B78
:103F4000D5C701F00001000C09012A51010A000146
:103F500011E0030A10E0010A0FE0040A0EE0030A70
:103F60000DE0010A0FE0030A11E00E0A35E0080A2D
:103F70003AE039D039D038D037D036D044B201D039
:103F8000448232D044A201D044922ED044B212D006
:103F900009012C6B2C51000198EC09F0000909E093
:103FA00009012C2B326F0001EAEC16F00901F2D75F
:103FB000000111D009012C6B2C5100017EEC0AF09C
:103FC000000909E009012C2B326F0001EAEC16F020
:103FD0000901F2D7000108D009012B5302E14492F4
:103FE00001D04482000100D044A202D0010E01D0D1
:103FF000000E016E000C09012B51010A000118E0AE
:10400000030A38E0010AD8B47BD0070AD8B4B4D088
:10401000010AD8B4E8D0030AD8B41CD1010AD8B434
:104020002FD10F0AD8B44ED1080AD8B45DD15CD1D3
:1040300009012D6BFF0E2C6F2D1110E02E6B2E51F0
:104040000B080BE3036A2E51CC0FE96E000E032020
:10405000EA6ED20EEF6E2E2BF2D70BD0036A000160
:104060008651CC0FE96E000E0320EA6ED20EEF6E81
:1040700009013CD109012C3D24D02D5322E12E6BA6
:104080002E510B081DE3036A2E51CC0F016E000E5A
:10409000032201C031F903C032F9300E2E25336FEF
:1040A0003E6B3D6FD20E3F6F000158EC11F032C9EC
:1040B000EAFF31C9E9FF01C0EFFF09012E2BE0D76C
:1040C0001ED0036A00018651CC0F016E000E032240
:1040D00001C031F903C032F9300E00018625090113
:1040E000336F3E6B3D6FD20E3F6F000158EC11F005
:1040F00032C9EAFF31C9E9FF01C0EFFF0901F6D07B
:1041000009012D6BFF0E2C6F2D111CE02E6B2E5113
:104110000B0817E3300E2E25316F036A2E51CC0F9A
:10412000E96E000E0320EA6EEFCF32F93F6B31C922
:104130003EF932C940F9000111EC12F009012E2BB1
:10414000E6D719D0300E000186250901316F036AC8
:1041500000018651CC0FE96E000E0320EA6EEFCF0E
:1041600032F909013F6B31C93EF932C940F900010A
:1041700011EC12F00901BAD0036A8651CC0FE96E36
:10418000000E0320EA6EEF50D1082BE3036A86513C
:10419000CC0FE96E000E0320EA6E010EEF24EF6EE5
:1041A000036A8651CC0FE96E000E0320EA6ED890A8
:1041B000EF3409012F6F306BD8B0302B30C902F0CB
:1041C0002FC901F00232013202320132023201C043
:1041D000BEFF02320230300B006EBD50CF0B00101C
:1041E000BD6E090183D0036A8651CC0FE96E000EC3
:1041F0000320EA6EEF5000082BE2036A8651CC0FD1
:10420000E96E000E0320EA6E010EEF5CEF6E036AAA
:104210008651CC0FE96E000E0320EA6ED890EF3481
:1042200009012F6F306BD8B0302B30C902F02FC985
:1042300001F00232013202320132023201C0BEFF0D
:1042400002320230300B006EBD50CF0B0010BD6E3D
:1042500009014CD0036A8651CC0FE96E000E032091
:10426000EA6EEFCF31F90901336B31C932F9050E2E
:10427000346F030E356F000107EC16F0090136D0DC
:10428000036A8651CC0FE96E000E0320EA6ED890C7
:10429000EF3409012F6F306BD8B0302B30C902F0EA
:1042A0002FC901F00232013202320132023201C062
:1042B000BEFF02320230300B006EBD50CF0B00103B
:1042C000BD6E14D009012D530EE12C51D2080BE321
:1042D000036A00018651CC0FE96E000E0320EA6EDE
:1042E0002CC9EFFF090102D0090100D0036A0001C7
:1042F0008651CC0FE96E000E0320EA6EEF50D20813
:1043000009E2036A8651CC0FE96E000E0320EA6EC3
:10431000D20EEF6E036A8651CC0FE96E000E0320B9
:10432000EA6E036AEFCF01F003C002F0000C09014E
:1043300034C903F03351332BD8B4342B376F03C057
:1043400038F935C939F93A6B03C03FF93E6F35C9C1
:1043500040F9000111EC12F0090134C903F03351A6
:10436000332BD8B4342B376F03C038F936C939F939
:104370003A6B03C03FF93E6F36C940F9000111ECBA
:1043800012F0000C2EC938F92DC937F932EC13F0B0
:1043900002C032F901C031F90901313D17D0323D77
:1043A00015D02EC934F92DC933F930C936F92FC9C2
:1043B00035F90001BCDF2EC938F92DC937F932ECC7
:1043C00013F002C032F901C031F9090131C901F01D
:1043D00032C902F0000134EF22F032C948F931C984
:1043E00047F9090E09014A6F360E496F34C94BF976
:1043F0004C6B35C94DF9000144EC15F009013553FA
:1044000001E0342B090E3D6F360E3C6F33C93EF987
:1044100034C93FF90001F8EC15F0000C09012A51EC
:10442000010A000112E0030A15E0010A22E0070A6E
:104430002BE0010A35E0030A3DE0010A54E00F0ACF
:1044400053E0080AD8B463D062D0010EA96F770E8A
:10445000A86F5ED009012E6B1C0E2D6F010E306F00
:10446000770E2F6F00018ED702C0A9F001C0A8F00F
:104470004FD00901346B1C0E336FA9C036F9A8C0A8
:1044800035F9000154DF44D0A951020808E303E1E3
:10449000A851700804E3190EA827000EA92338D0EC
:1044A000A95303E1A851AF0804E2190EA85F000E5A
:1044B000A95B2ED0A83509012D6F0001A93509018E
:1044C0002E6F2D372E372D372E37F80E2D172EC97C
:1044D00032F92DC931F9040E336F346F030E356F85
:1044E00000017BDF15D014D009012C5303E12B51BF
:1044F000AE080BE22C51020808E303E12B517108CE
:1045000004E32CC9A9F02BC9A8F0000101D000D008
:10451000A95303E1A851AE0808E2A951010809E234
:10452000FF0A03E1A851710804E2010EA96F770E9A
:10453000A86FA8C001F0A9C002F0000CA092000C66
:1045400009012751010A000119E0030A1BE0010AD1
:1045500047E0070A50E0010AD8B476D0030AD8B47D
:104560009BD0010AD8B4BED00D0AD8B4DED0010A5F
:10457000D8B402D10B0AD8B402D101D1430E08013C
:10458000F26FFFD009013E6B0F0E3D6F430E3F6F80
:10459000000158EC11F001C0F2F809013E6BF2C8BD
:1045A0003DF9406B040E3F6F0001ABEC11F001C010
:1045B00028F9020E09010124016E000E0220036E8B
:1045C0000150D60FE96E070E0320EA6EECCF03F020
:1045D000ED52EFCF84F0000103C085F00801D1D087
:1045E00009013F6B0F0E3E6FF2C840F9000111EC5C
:1045F00012F00801C6D00801F251450824E3010E6B
:10460000F22709013E6BF2C83DF9406B040E3F6F83
:104610000001ABEC11F001C028F9020E09010124E0
:10462000016E000E0220036E0150D60FE96E070ED8
:104630000320EA6EECCF03F0ED52EFCF84F00001DF
:1046400003C085F008019DD00801F25324E0010E5B
:10465000F25F09013E6BF2C83DF9406B040E3F6FFB
:104660000001ABEC11F001C028F9020E0901012490
:10467000016E000E0220036E0150D60FE96E070E88
:104680000320EA6EECCF03F0ED52EFCF84F000018F
:1046900003C085F0080175D009013E6BF2C83DF9F1
:1046A000406B040E3F6F0001ABEC11F002C029F922
:1046B00001C028F9D60E09010124E96E070E022077
:1046C000EA6EECCF2BF9ED52EFCF2AF92BC933F973
:1046D0002AC932F9040E346F356F000107EC16F069
:1046E00008014FD009013E6BF2C83DF9406B040E42
:1046F0003F6F0001ABEC11F001C028F9020E090177
:104700000124016E000E0220036E0150D60FE96EE7
:10471000070E0320EA6EECCF03F0ED52EFCF84F0EA
:10472000000103C085F008012CD0850EB16E09018F
:104730003E6BF2C83DF9406B040E3F6F0001ABECDD
:1047400011F001C028F9020E09010124016E000ECA
:104750000220036E0150D60FE96E070E0320EA6EA9
:10476000ECCF2BF9ED52EFCF2AF92BC9B3FF2AC9B1
:10477000B2FFA082080105D0E1DE080102D00801E5
:1047800000D0F251460802E2430EF26F09013E6B7F
:10479000F2C83DF9406B040E3F6F0001ABEC11F025
:1047A00002C029F901C028F9020E09010124016E95
:1047B000000E0220036E0150D60FE96E070E032093
:1047C000EA6EEFCF01F0E92AEF50E906026E000130
:1047D000B0EF25F009012A51010A000111E0030A96
:1047E00010E0010A0FE0040A0EE0030A0DE0010ADE
:1047F0000FE0030A11E00E0A35E0080A3EE03DD062
:104800003DD03CD03BD03AD044B401D0448436D0E3
:1048100044A401D0449432D044B412D009012C6B8A
:104820002C51000167EC0AF0000909E009012C2B6A
:10483000326F0001EAEC16F00901F2D7000111D045
:1048400009012C6B2C51000195EC0AF0000909E0DC
:1048500009012C2B326F0001EAEC16F00901F2D7A6
:1048600000010CD009012B5302E0010E01D0000E13
:104870004494E8B04484000101D000D044A402D0A4
:10488000010E01D0000E016E000C09012E5302E052
:10489000010E01D0000E8A92E8B08A820001000C5D
:1048A00009012D6B2E6B000114EC1EF001C02CF9D8
:1048B00009012A51010A000112E0030A11E0010A6C
:1048C00010E0040A0FE0030A18E0010A1DE0030AE1
:1048D00022E00E0A5BE0080AD8B465D064D064D048
:1048E00063D062D044A802D0010E01D0000E0901AD
:1048F0002D6F2E6F0001C9DF57D009012C5103081D
:1049000001E14488000150D009012C51030801E164
:104910004498000149D009012C51030826E144B80C
:1049200012D02D6B2D51000198EC09F0000909E01F
:1049300009012D2B326F0001EAEC16F00901F2D7C4
:10494000000111D009012D6B2D5100017EEC0AF000
:10495000000909E009012D2B326F0001EAEC16F085
:104960000901F2D7000111D009012D6B2D51000171
:10497000F1EC0AF0000909E009012D2B326F00016A
:10498000EAEC16F00901F2D700010ED009012C5112
:10499000030807E12B5302E1449803D02B2D01D0EB
:1049A0004488000101D000D044A802D0010E01D0FB
:1049B000000E016E000C09012A51010A000111E0EC
:1049C000030A11E0010A10E0040A0FE0030A0EE0F6
:1049D000010A10E0030A12E00E0A36E0080A3BE082
:1049E0003AD0449C39D038D037D036D044BC01D0EE
:1049F000448C32D044AC01D0449C2ED044BC12D064
:104A000009012C6B2C51000195EC0AF0000909E01A
:104A100009012C2B326F0001EAEC16F00901F2D7E4
:104A2000000111D009012C6B2C510001ACEC0AF0F3
:104A3000000909E009012C2B326F0001EAEC16F0A5
:104A40000901F2D7000108D009012B5302E1449C6F
:104A500001D0448C000100D044AC02D0010E01D042
:104A6000000E016E000C020E09012D6F000122ECF8
:104A700016F0020E09012D6F0001F3EC16F0020E84
:104A800009012D6F000167EC17F0020E0901276F75
:104A90000001CBEC19F0020E09012A6FFF0E2B6FFB
:104AA000000133EC1AF0020E09012A6F00016EECCE
:104AB0001BF0020E09012A6F2B6B000134EC1CF075
:104AC000070E09012A6F2B6B000134EC1CF0020E5B
:104AD00009012A6F2B6B000148EC1DF0070E09013C
:104AE0002A6F2B6B000148EC1DF0020E09012D6F9F
:104AF0002E6B000114EC1EF0020E09012A6F2B6BC5
:104B00000001CBEC1EF0020E09012A6F2B6B000195
:104B10002BEC1FF0020E09012A6F2B6B0001A4EC95
:104B20001FF0020E09012B6F2D6BFF0E2C6F000181
:104B3000FBEC1FF0070E09012B6F2D6BFF0E2C6F86
:104B40000001FBEC1FF0020E09012A6F2C6BFF0E17
:104B50002B6F000163DC020E0901276F0001F0D406
:104B6000020E09012A6FFF0E2B6F000133DE020EC9
:104B700009012A6F2B6B000193DE070E09012A6FD2
:104B80002B6B00018DDE020E09012A6F2B6B0001D9
:104B900012DF000C8A9A91868A88919C8B826A9D8A
:104BA0006A9F4192496A476A070E09012A6F2B6B77
:104BB0000001CBEC1EF0000C706B6F6B8E8E8A9434
:104BC000736B6C6B726B716BFFEF63F06B6B01EF70
:104BD00064F0536A656B666B03EF64F00701416B29
:104BE0000401196B1A6B146BABCF22F9ABA202D084
:104BF000800EAB6EE86A9EBAE82AAECFE8FF9D8AC7
:104C0000900EAB6E000105EF64F04C6A07013F6B3C
:104C1000406B3C6B6BCF22F96BA802D0800E6B6EA1
:104C2000E86AA4BAE82A6ECFE8FFA38A900E6B6EFA
:104C3000000107EF64F00901386BE00E376F0001E7
:104C400032EC13F002C02CF901C02BF909012A51F2
:104C5000F80F38E2080F000168EF26F0090132D0A2
:104C6000090130D009012ED009012CD009012AD028
:104C7000090128D0090126D009012B3D03D02C3D84
:104C800001D00DD02CC933F92BC932F9030E346F82
:104C9000050E356F000107EC16F011D009012D6BE0
:104CA0002D51000134EC08F0000909E009012D2B19
:104CB000326F0001EAEC16F00901F2D70001090198
:104CC00001D009012BC901F02CC902F00001000C30
:104CD000F2CF21F0F29CF29EE824F76AF736010F3A
:104CE000F66E4D0EF722000EF86EFB6E0A00F550C0
:104CF000FA6E0800F55021BCF28C21BEF28EF96EDE
:104D00005C4C604C644C684C6C4C704C784C744CF3
:104D10000901226B2A6B00018EDF02C024F901C059
:104D200023F90901226BD8902235036AF2CF25F9C5
:104D3000F29CF29E0001CBEC06F00900F5CF03F0E7
:104D4000090125BDF28C25BFF28E03101BE0D8901F
:104D50002235036AF2CF25F9F29CF29E0001CBECDA
:104D600006F00900F5CF03F0090125BDF28C25BF3F
:104D7000F28E235D05E10350245D02E1438203D0FE
:104D8000222BD1D74392000109EF64F00901306B67
:104D9000530E316F3151305D3DE23051315D006E67
:104DA000D890003200503025326F3E6B32C93DF949
:104DB000406B0C0E3F6F0001ABEC11F002C034F9F8
:104DC00001C033F9060E09010124016E000E022014
:104DD000036E0150F2CF35F9F29CF29E03C0F7FF4B
:104DE0000001C2EC04F00900F5CF03F0090135BD64
:104DF000F28C35BFF28E016E2F51035C07E303E1A5
:104E000001502E5D03E232C931F903D0010E322583
:104E1000306FC0D7010E305D036A016E03C002F02F
:104E20000001A2EF27F086510A082DE109013E6B2F
:104E30002EC93DF9406B0C0E3F6F0001ABEC11F039
:104E400002C030F901C02FF9040E09010124016EDE
:104E5000000E0220036E0150F2CF31F9F29CF29E57
:104E600003C0F7FF0001C2EC04F00900F5CF03F026
:104E7000090131BDF28C31BFF28E016E03C002F028
:104E800059D032D000018651090803E08651080844
:104E90002BE109013E6B2EC93DF9406B0C0E3F6FB3
:104EA0000001ABEC11F002C030F901C02FF9020E85
:104EB00009010124016E000E0220036E0150F2CFA1
:104EC00031F9F29CF29E03C0F7FF0001C2EC04F03E
:104ED0000900F5CF03F0090131BDF28C31BFF28E2C
:104EE000016E03C002F026D009013E6B2EC93DF9C8
:104EF000406B0C0E3F6F0001ABEC11F002C030F9BB
:104F000001C02FF902C003F009010150F2CF31F9BD
:104F1000F29CF29E02C0F7FF0001C2EC04F009000F
:104F2000F5CF03F0090131BDF28C31BFF28E016E75
:104F300003C002F00001A7EF27F02CC92FF92BC9FD
:104F40002EF924D701C02DF92DC92EF96CD70250A6
:104F5000000C09012551F00B03E007014D6B09011D
:104F60000F0E251707014E510901255D03E00701CA
:104F70004D6B09014952D8A47ED107014D51000162
:104F80001BE0010A3FE0030AD8B46BD1010AD8B490
:104F900068D1070AD8B465D1010AD8B462D1030A2E
:104FA000D8B45FD1010AD8B45CD10F0AD8B459D1B2
:104FB000010AD8B45AD159D1428244A420D043B076
:104FC0001ED041A21CD00901255107014E5DD8A475
:104FD00002D0000114D00001875304E1535202E1D2
:104FE0000B0E536E2C6AF2BC2C8CF29CF2BE2C8EF3
:104FF000F29E39EC0EF02CBCF28C2CBEF28E43905B
:1050000025C94EF709012C6B640E2B6F000195DF4B
:1050100002C003F0015001014251025CD8A020D12E
:1050200004E10150415DD8B01BD107014E51010A86
:10503000000115E0030A1BE0020A21E0030A27E051
:10504000070A2DE0010A32E0030A38E0010A3EE0D7
:105050000F0A44E0010A4AE0030A50E057D0200E4C
:105060000901276F286B296B010E2A6F57D0400E5C
:105070000901276F286B296B800E2A6F4FD0800E95
:105080000901276F286B296B020E2A6F47D0080E83
:105090000901276F286B296B400E2A6F3FD0040E41
:1050A0000901276F286B296B2A6F38D0020E09017E
:1050B000276F286B296B200E2A6F30D0010E090153
:1050C000276F286B296B080E2A6F28D00901276BE0
:1050D000080E286F010E296F2A6B20D00901276B5B
:1050E000040E286F020E296F2A6B18D00901276B56
:1050F000020E286F040E296F2A6B10D00901276B4E
:10510000010E286F080E296F2A6B08D00901276B42
:10511000010E286F080E296F2A6B00D007014E512F
:105120000A0802E1010E01D0000E8A90E8B08A80E0
:10513000020E09012B6FC69A2B2D03D0300EC66EBE
:1051400002D0320EC66EC76AC68A0D0E006E002EE1
:10515000FED7F29CF29EF2BEFDD79198919E020E70
:10516000006E002EFED700002AC931F9C9CF32F9EE
:1051700031C9C9FFC7A0FED7C9CF32F9326B32514E
:10518000010802E3322BFBD729C931F9C9CF32F923
:1051900031C9C9FFC7A0FED7C9CF32F9326B32512E
:1051A000010802E3322BFBD728C931F9C9CF32F904
:1051B00031C9C9FFC7A0FED7C9CF32F9326B32510E
:1051C000010802E3322BFBD727C931F9C9CF32F9E5
:1051D00031C9C9FFC7A0FED7C9CF32F9326B3251EE
:1051E000010802E3322BFBD7020E006E002EFED721
:1051F0000000918E9188C00EF212010E2B6FC69A9C
:105200002B2D03D0300EC66E02D0320EC66EC76A8A
:10521000C68A0D0E006E002EFED7265311E0000147
:10522000A451A511D8B402D009010AD0895110089F
:10523000D8A402D0090104D0896BA56B7D0EA46FA0
:10524000000186510B0808E3070E09012B6F2D6B37
:105250002C6B0001FBEC1FF0020E07014D6F0101EA
:1052600009D007014D2B010105D0429207014D6B7A
:10527000010100D009010001000C0901236B0A0E95
:105280000701A4250901246F2435006E0036FC0EA9
:105290000016C250C30B0010C26E270E006E002E07
:1052A000FED700D0C282C2B2FED7C430036EC33074
:1052B000026E0332023202C022F922515A0832E24F
:1052C0002251DA0806E2040E0701A4250901236F22
:1052D00029D02251C00806E2080E0701A4250901C1
:1052E000236F20D02251A60806E20C0E0701A42548
:1052F0000901236F17D022518D0806E2100E070115
:10530000A4250901236F0ED02251730806E2140E62
:105310000701A4250901236F05D0180E0701A42554
:105320000901236F84AC01D042880701A45308E12E
:1053300042A806D084BC04D01C0E0901236F0701CB
:10534000A25100010AE0010A14E0030A33E0010A55
:105350005CE0070AD8B471D080D009012351FC0B5E
:1053600007E023C946F00701A36B010EA26F0901F4
:1053700078D00701A32BA3510C081AE1090123518E
:10538000465C04E00701A26B13D00901036A2351B4
:10539000850FE96E070E0320EA6EEF5206E1010E5B
:1053A000456E040E0701A26F03D0020E0701A26F23
:1053B000090157D00701A32BA351FC0815E1020EE8
:1053C000456E036A09012351850FE96E070E03201C
:1053D000EA6EEFA205D00701A36B030EA26F03D004
:1053E000040E0701A26F0FD04650030BA45D0BE122
:1053F00009012351465CD8A402D0070104D0010E54
:10540000456E0701A26B09012CD00701A32BA35104
:105410001E0804E1030E456EA36B0DD04650030B2E
:10542000A45D09E109012351465CD8A402D007011B
:1054300002D00701A26B090114D04650030B0701EB
:10544000A45D09E109012351465CD8A402D00701FB
:1054500002D00701A26B090104D00701A26B090168
:1054600000D00701A42BA451020801E2A46B0001A3
:105470001BEF64F00901245107083DE303E12351C8
:10548000E80839E3245103081DE303E1235106082A
:1054900019E32451010807E303E12351380803E32A
:1054A000010E016E5ED02451020808E303E123518E
:1054B0003E0804E3020E016E54D003D0000E016ECC
:1054C00050D018D02451040807E303E123512608E3
:1054D00003E3030E016E45D02451050808E303E100
:1054E00023519D0804E3040E016E3BD003D0050E4A
:1054F000016E37D034D024510C081DE303E1235151
:10550000B10819E32451090807E303E12351850891
:1055100003E3060E016E25D024510B0808E303E1D6
:1055200023513A0804E3070E016E1BD003D0080E86
:10553000016E17D014D024510D0807E303E1235165
:10554000AA0803E30C0E016E0CD02451100807E3E7
:1055500003E123511C0803E3090E016E02D00A0E79
:10556000016E0001CEEF2AF00F0E09012817285115
:105570000001865D06E0090128510F0B0001866FCE
:105580004282000C0101385303E13751C80831E26F
:1055900038C124F937C123F900016CD701C022F9C1
:1055A00007014F510901225D21E1429422510C086B
:1055B00004E143A202D0090E226F22510C080EE131
:1055C0000701502B5051010807E24284020E506F30
:1055D0000F0E0001866F070108D009010701506B0B
:1055E00022C928F90001C0DF0701090122C94FF7CC
:1055F0000101386B376B00011DEF64F08B800D0EDD
:105600000901236F0001C0EC18F00901236B0001B0
:10561000C0EC18F0010E0901236F0001C0EC18F076
:10562000020E0901236F0001C0EC18F0030E0901FE
:10563000236F0001C0EC18F0060E0901236F000172
:10564000C0EC18F0080E0901236F0001C0EC18F03F
:10565000090E0901236F0001C0EC18F08B906FEF69
:105660002DF00901286B530E296F2951285D3DE269
:105670002851295D006ED8900032005028252A6FED
:105680003E6B2AC93DF9406B0C0E3F6F0001ABEC3D
:1056900011F002C02CF901C02BF9040E09010124FC
:1056A000016E000E0220036E0150F2CF2DF9F29C24
:1056B000F29E03C0F7FF0001C2EC04F00900F5CF31
:1056C00003F009012DBDF28C2DBFF28E016E275122
:1056D000035C07E303E10150265D03E22AC929F9CF
:1056E00003D0010E2A25286FC0D7010E285D016E58
:1056F000000117EF2CF00901286B530E296F295177
:10570000285D3DE22851295D006ED890003200509E
:1057100028252A6F3E6B2AC93DF9406B0C0E3F6F5E
:105720000001ABEC11F002C02CF901C02BF9020E04
:1057300009010124016E000E0220036E0150F2CF18
:105740002DF9F29CF29E03C0F7FF0001C2EC04F0B9
:105750000900F5CF03F009012DBDF28C2DBFF28EAB
:10576000016E2751035C07E303E10150265D03E26C
:105770002AC929F903D0010E2A25286FC0D7010EA6
:10578000285D016E000125EF2CF00901286B530EF6
:10579000296F2951285D39E22851295D006ED89082
:1057A0000032005028252A6F3E6B2AC93DF9406B14
:1057B0000C0E3F6F0001ABEC11F002C02CF901C0E0
:1057C0002BF902C003F009010150F2CF2DF9F29C30
:1057D000F29E02C0F7FF0001C2EC04F00900F5CF11
:1057E00003F009012DBDF28C2DBFF28E016E275101
:1057F000035C07E303E10150265D03E22AC929F9AE
:1058000003D0010E2A25286FC4D7010E285D016E32
:1058100000012DEF2CF0540E0901256F0001865177
:105820000A0808E124C927F923C926F91AD701C0B3
:1058300025F915D08651090803E08651080808E1CA
:1058400024C927F923C926F956D701C025F907D05D
:1058500024C927F923C926F998D701C025F90901D8
:1058600025C901F00001000C09012A6B2B6B000116
:1058700033EC1AF001C022F9D890FD3101013E6FDE
:105880000001FC3101013D6F01C140F100C13FF158
:10589000000186510A080EE10101405303E13F5126
:1058A000640805E2640E3F5F000E405B02D0406B6F
:1058B0003F6B0001D890010140333F333EC13EF9B8
:1058C0003DC13DF90901406B22C93FF90001ABEC34
:1058D00011F002C03EF101C03DF101013E333D3304
:1058E0003E333D333E333D333E333D333E333D3334
:1058F000070E3E1740C13EF93FC13DF90901406B1B
:1059000022C93FF90001ABEC11F002C040F101C027
:105910003FF1010140333F3340333F3340333F33A6
:1059200040333F3340333F33070E40173EC124F925
:105930003DC123F900016FDF01C03BF109013E6B5E
:105940003BC13DF9406B0C0E3F6F0001ABEC11F019
:1059500002C024F901C023F9060E09010124016ED9
:10596000000E0220036E0150F2CF25F9F29CF29E48
:1059700003C0F7FF0001C2EC04F00900F5CF03F00B
:10598000090125BDF28C25BFF28E0101456F03C0D0
:1059900046F140C124F93FC123F900013CDF01C0B9
:1059A0003CF109013E6B3CC13DF9406B0C0E3F6F71
:1059B0000001ABEC11F002C024F901C023F9060E7E
:1059C00009010124016E000E0220036E0150F2CF86
:1059D00025F9F29CF29E03C0F7FF0001C2EC04F02F
:1059E0000900F5CF03F0090125BDF28C25BFF28E29
:1059F0000101476F03C048F13D510801FA27010139
:105A00003E510801FB2301013F510801FC27010120
:105A100040510801FD2309013E6B3BC13DF9406B3C
:105A20000C0E3F6F0001ABEC11F002C024F901C075
:105A300023F9060E09010124016E000E0220036EF7
:105A40000150F2CF25F9F29CF29E03C0F7FF00014E
:105A5000C2EC04F00900F5CF03F0090125BDF28C7A
:105A600025BFF28E0801FE270350FF23F92BF951C1
:105A700004082BE1FB310101426F0801FA310101F9
:105A8000416F423341333F0E42170801FD3101019E
:105A9000446F0801FC310101436F443343333F0E2F
:105AA00044170801FB6BFA6BFD6BFC6BF96BFF3164
:105AB00001014C6F0801FE3101014B6F4C334B3338
:105AC0003F0E4C170801FF6BFE6B0001FD6BFC6B7A
:105AD0000101016B006B000170EF2DF08FD5C4D672
:105AE00031EF64F001014A6B496B000173A504D0EA
:105AF00084B802D041B207D00901016B006B0701E5
:105B00004899419E000173B703D00901036B026BF2
:105B10000101465304E145511808D8B0EBD040517B
:105B20003E5D3FE303E13D513F5D3BE23F513D259B
:105B30000901266F010140513E210901276F3E6F87
:105B400026C93DF9406B140E3F6F0001ABEC11F01C
:105B500002C023F901C022F901013F513D5D090155
:105B6000246F010140513E590901256F23C951F9A4
:105B700022C950F925C953F924C952F9000121EC71
:105B800015F0010E09010124286F000E0220296F73
:105B9000D890293101014A6F090128310101496F6B
:105BA00004D0010E4A6FF40E496F84B84ED041A262
:105BB0004CD009012C6B640E2B6F00019DEC27F07B
:105BC0000250036E0101405D13E303E13F51015CAC
:105BD0000FE2000173850901002BD8B4012B01539A
:105BE00006E10051080803E3016B090E006F16D0AF
:105BF00009012C6B3C0E2B6F00019DEC27F002502D
:105C0000036E0101405D0BE303E13F51015C07E2DC
:105C1000000173850901002BD8B4012B01014A53FF
:105C200003E14951B40811E284AA0FD00001738541
:105C30000901002BD8B4012B015306E100510808DB
:105C400003E3016B090E006F010109013E6BBFC048
:105C50003DF9406B0C0E3F6F0001ABEC11F002C040
:105C600027F901C026F9060E09010124016E000E74
:105C70000220036E0150F2CF28F9F29CF29E03C07D
:105C8000F7FF0001C2EC04F00900F5CF03F00901B1
:105C900028BDF28C28BFF28E226F03C023F9235156
:105CA0000101465D25E308E145510901225DD8A0C7
:105CB00002D001011DD001010901042B0451080883
:105CC00005E200017387080E0901046F022BD8B4A6
:105CD000032B035303E10251080809E20001708518
:105CE00046C17DF045C17CF00901036B026B02D017
:105CF0000901046B070148A904D00901002BD8B49D
:105D0000012B0901015303E1005120080EE2418EED
:105D100000016F8F40C17FF03FC17EF00901016B30
:105D2000006B070148990DD00901015303E10051AF
:105D3000080805E207014889418E03D00901419E08
:105D4000070100013FEF32F0036A090123511A0FE6
:105D5000E96E010E0320EA6EEFCF25F92551030805
:105D600046E2D8902435036A2E0F016E010E0322FD
:105D700003C027F9D8902335036AFA0FE96E000EA5
:105D80000320EA6EECCF29F9ED52EFCF28F9020E8D
:105D900028252A6F000E29212B6F2B31036E2A3103
:105DA000026E033202323F0E031627C9EAFF01C01A
:105DB000E9FF03C0ECFFED5202C0EFFFD89023359E
:105DC000036AFA0FE96E000E0320EA6EEC6AED52E8
:105DD000EF6A036A23511A0FE96E010E0320EA6E7F
:105DE000EF6A2551040803E1010E016E02D0000E96
:105DF000016E0001000C000E010136B1010E090117
:105E0000226F020E236F246B00019EDF09012251D5
:105E1000011001013691E8B036813683000E36B5A7
:105E2000010E0901226F060E236F020E246F00017E
:105E30008BDF09012251011001013695E8B036854A
:105E4000368736510F0A42E10901122B125104081C
:105E500013E14B6A226B225100016AEC09F0000940
:105E600009E00901222B326F0001EAEC16F009016A
:105E7000F2D7000129D0090112510C0805E12FC108
:105E8000D9F02EC1D8F020D0125113081DE241865E
:105E900000016C6B0901126B12510C0815E3D890CC
:105EA0001235036AFA0FE96E000E0320EA6EEC6AFF
:105EB000ED52EF6A036A12511A0FE96E010E0320C8
:105EC000EA6EEF6A122BE8D70101366B000143EF4F
:105ED00032F073B105D00901086B076B096B000143
:105EE00015C123F914C122F949500208D8A4CBD016
:105EF000090122510B2723510C23235303E1225183
:105F00003C0825E201013E53D8B402D009011FD05C
:105F10003D516308D8B002D0090119D009010E51D2
:105F200004080DE3428200018651F0090901246F43
:105F3000256F266B0001A9EC27F007D009010001AD
:105F40006F89B7C079F0B6C078F002D009010E6B46
:105F500009010A2B0A510308D8B093D0020E0B2571
:105F6000246F000E0C21256F25310001B76F090148
:105F700024310001B66FB733B6333F0EB717B751B0
:105F800001080AE2FF0A03E1B651F50805E26F894C
:105F9000B7C079F0B6C078F0B751010813E2FF0A34
:105FA00003E1B6519E080EE2090109513B0808E2DF
:105FB00000016F89B7C079F0B6C078F003D009014D
:105FC000092B0001B75101081BE2FF0A03E1B6519A
:105FD000620816E273810901085101080DE2FF0A07
:105FE00003E10751700808E200016F89B7C079F03A
:105FF000B6C078F005D00901072BD8B4082B0001F2
:1060000009010C6B0B6B0A6B3E6B3BC13DF9406B9E
:106010000C0E3F6F0001ABEC11F002C025F901C07E
:1060200024F9080E09010124016E000E0220036EFE
:106030000150F2CF26F9F29CF29E03C0F7FF000157
:10604000C2EC04F00900F5CF03F0090126BDF28C83
:1060500026BFF28E016E0001B751035C13E303E12A
:106060000150B65D0FE209010D2B0D51320808E217
:1060700000017087B7C083F0B6C082F003D0090179
:106080000D6B000107D009010A6B0C6B0B6B000153
:10609000B76BB66B0101156B146B276B000149EFF1
:1060A00032F001011A51040857E1020E0001FA25ED
:1060B0000901246F000E0001FB210901256F253124
:1060C000276F2431266F273326333F0E271727C922
:1060D0003EF926C93DF9406B050E3F6F0001ABEC60
:1060E00011F002C0B3F001C0B2F044AA04D0080E0F
:1060F000B36FC00EB26F100EB2250901246F000EEF
:106100000001B3210901256F2531236F2431226F4E
:1061100023332233233322332333223323332233D3
:10612000070E231741A20CD023530AE1225127085E
:1061300007E30001708B23C97BF022C97AF00901C3
:10614000235303E122515A0807E200016F8D23C94E
:106150007BF022C97AF009010001FB6BFA6B0101A7
:106160001A6B00014FEF32F073B303D00901066BD5
:10617000056B01011C510408D8A470D0020E000167
:10618000FE250901266F000E0001FF210901276F7E
:1061900027310001FF6F090126310001FE6FFF3337
:1061A000FE333F0EFF1741A206D001012AA507D0FA
:1061B0002CA505D00001FFC0D9F0FEC0D8F0000129
:1061C000D851FE5D006ED951FF5900C024F9090174
:1061D000256F44AA0BD084A806D0020E0001D96F07
:1061E000D86B05D00901256BB60E246F0001B16B89
:1061F000B06B090125BF32D0255303E124510008BB
:106200002DE225C93EF924C93DF9406B130E3F6FBD
:106210000001ABEC11F001C0B0F002C0B1F0800E93
:10622000B025000E0001B1210901226F236B235319
:1062300003E12251140812E2000173830901052BC6
:10624000D8B4062B065303E10551020807E200010A
:106250006F8123C975F022C974F009010001FF6B39
:10626000FE6B01011C6B000155EF32F00101205162
:10627000200839E1100E06250901226F000E0101E8
:1062800007210901236F23310001AF6F090122317A
:106290000001AE6FAF33AE33AF33AE33AF33AE3397
:1062A000AF33AE33070EAF17AFC03EF9AEC03DF906
:1062B0000901406B7D0E3F6F0001ABEC11F0800EC9
:1062C00009010124000E0220E8CFAAF00001AB6B07
:1062D000AB5303E1AA515A0805E26F85ABC077F0D2
:1062E000AAC076F00101076B066B206B00015BEF23
:1062F00032F009012D512F19800B316F2DAF05D0D0
:106300002C1F2D1F2C2BD8B42D2B2FAF05D02E1FBB
:106310002F1F2E2BD8B42F2B016A026A006A036A42
:106320002F5102E12E5118E0100E306FD8902C370B
:106330002D37003603362F51035C02E12E51005CED
:1063400007E32E51005ED8A003062F51035ED880CC
:1063500001360236302FEAD731AF05D0011E021EBA
:10636000012AD8B4022A0001E5EF31F0D85303E145
:10637000D953D8B47FD041A27DD044BA7BD0D85174
:10638000DE5D006ED951DF5900C022F90901236F8B
:1063900023C93EF922C93DF9406B130E3F6F00013E
:1063A000ABEC11F002C029F901C028F9800E0901F7
:1063B00001242A6F000E02202B6F2D6F2AC92CF9A1
:1063C000010E2F6F2E6B000194D702C025F9090131
:1063D00001C024F9DBC03EF9DAC03DF9406B050E7F
:1063E0003F6F0001ABEC11F0100E090101242A6F80
:1063F000000E02202B6F2B31276F2A31266F273397
:106400002633273326332733263327332633070E05
:10641000271727C93EF926C93DF925C940F924C9DE
:106420003FF90001ABEC11F0010145510901015C9C
:10643000006E010146510901025800C04DF10101F1
:106440004E6F4EBF15D04E51010812E2FF0A03E114
:106450004D5158080DE209010F2B0F51080807E2B2
:10646000000170834EC181F04DC180F0090102D05E
:1064700009010F6B00019DEF32F072EF2DF04850D3
:10648000100802E1B8D453D00101275303E0000102
:1064900020D501011A51030803E2000102D60101CF
:1064A0001C51030803E200015FD6010120511F08BF
:1064B00003E20001DBD601012351070837E2235133
:1064C00008082EE1040E0C250901226F000E0101BF
:1064D0000D210901236F23310001B96F0901223118
:1064E0000001B86FB933B833B933B8331F0EB917D9
:1064F000040E01010A250901226F000E01010B2182
:106500000901236F23310001BB6F09012231000112
:10651000BA6FBB33BA33BB33BA331F0EBB1701019B
:106520000D6B0C6B0B6B0A6B236B226B000141A292
:1065300003D088A001D0708919D735EF64F0010E1F
:1065400007013E253D5D0AE01C0E3E25E96E040E66
:10655000EA6ED8B0EA2A26C9EFFF3E2BA3880001D5
:10656000C8EF44F00901296B2A6B28512807000A5B
:1065700029E007014451442B036A1C0FE96E060E03
:106580000320EA6EEFCF01F0300E015C09012B6FA2
:106590002B51090805E229C901F02AC902F016D0D9
:1065A0002AC93EF929C93DF9406B0A0E3F6F000127
:1065B000ABEC11F009012B510124296F000E0220D0
:1065C0002A6FD3D729C901F02AC902F00001000CB3
:1065D00009012E6B2BC948F92AC947F9090E4A6FE0
:1065E0002F0E496F2CC94BF9010E4C6F2DC94DF977
:1065F000000144EC15F0036A09012E512F0FE96EDA
:10660000090E0320EA6EEF521AE02E512E2B036A78
:106610002F0FE96E090E0320EA6EEFCF3AF93AC95F
:106620003BF907014351432B036AAC0FE96E060E99
:106630000320EA6E3BC9EFFF0001DDD70901010E1F
:10664000016E0001000C07014351432B036AAC0F9C
:10665000E96E060E0320EA6E3B0EEF6E4351432BAC
:10666000036AAC0FE96E060E0320EA6EEF6A0901B9
:106670002C6B036A2C51AC0FE96E060E0320EA6EF8
:10668000EF522BE00701435109012C5D26E22C510A
:106690008F0823E3010E07013E253D5D1BE01C0E24
:1066A0003E25016E040E036ED8B0032A090103C013
:1066B0002EF9036A2C51AC0FE96E060E0320EA6E28
:1066C000EFCF2FF92EC9EAFF01C0E9FF2FC9EFFF75
:1066D00007013E2B09012C2BCCD7A3880001000C0D
:1066E0000701465105080EE1010E0901286F00015E
:1066F00039DF01C026F909012651020802E326C943
:106700004CF00701465104080BE109012B6B4CC00A
:106710002AF9010E2C6F2D6B00015ADF94DF07015F
:10672000000136EF45F007014651070824E1030E4A
:106730000901286F000116DF02C027F901C026F900
:10674000080E09012B6F27C92DF926C92CF9000164
:10675000FBEC1FF0030E09012B6F2D6B2C6B00015E
:10676000FBEC1FF0070E09012B6F2D6B2C6B00014A
:10677000FBEC1FF007014651040817E109012B6BE0
:106780002D6B2C6B0001FBEC1FF002C027F901C040
:1067900026F927C92BF926C92AF9030E09012C6FFE
:1067A0002D6B000115DF4FDF070100013EEF45F0C3
:1067B0000901266B276B07014651080828E1040EE2
:1067C0000901286F0001CEDE040E090101242A6FA1
:1067D000000E02202B6F2B31276F2A31266F2733B3
:1067E0002633273326331F0E2717080E2A6F27C993
:1067F0002CF926C92BF900010EEC22F0030E090139
:106800002A6F2C6B2B6B00010EEC22F00701465116
:1068100004081DE109012A6B2C6B2B6B00010EECA7
:1068200022F009010134266F0234276F26372737FB
:1068300026372737F80E261727C92BF926C92AF934
:10684000040E2C6F2D6B0001C3DEFDDE070100017D
:1068500046EF45F073A122D00901326B8A0E316FE9
:10686000336B070E346F0001C7EC17F00901276B7B
:1068700027510001D1EC0BF0000909E00901272B99
:10688000326F0001EAEC16F00901F2D70001010EA7
:106890006D6FA9C0BDF0A8C0BCF0A5D073A322D075
:1068A0000901326B8A0E316F336B070E346F0001B2
:1068B000C7EC17F00901276B275100018CEC0BF096
:1068C000000909E00901272B326F0001EAEC16F0FC
:1068D0000901F2D70001020E6D6FA9C0BDF0A8C07A
:1068E000BCF081D073A508D0030E6D6FA9C0BDF0B8
:1068F000A8C0BCF081D077D073A722D00901326B39
:106900008A0E316F336B070E346F0001C7EC17F03E
:106910000901276B275100015BEC0CF0000909E02D
:106920000901272B326F0001EAEC16F00901F2D7BA
:106930000001040E6D6FA9C0BDF0A8C0BCF053D01B
:1069400073A922D00901326B8A0E316F336B070EA7
:10695000346F0001C7EC17F00901276B27510001C4
:1069600044EC0CF0000909E00901272B326F00010B
:10697000EAEC16F00901F2D70001050E6D6FA9C00F
:10698000BDF0A8C0BCF02FD073AF21D00901326B8D
:106990008A0E316F336B070E346F0001C7EC17F0AE
:1069A0000901276B27510001CEEC0CF0000909E02A
:1069B0000901272B326F0001EAEC16F00901F2D72A
:1069C0000001080E6D6FFF0EBD6FBC6F0CD009018A
:1069D000326B8A0E316F336B070E346F0001C7ECD8
:1069E00017F06D6B09D00801F651080802E088C065
:1069F000F6F8080E0001886F000C010E6D5DF80FAF
:106A00000FE2080F1BEF35F073910AD0739308D093
:106A1000739506D0739704D0739902D0739F00D0FA
:106A20008851080802E1F6C888F0BD6BBC6B73534F
:106A300001E010DF000CF2CF21F0F29CF29EE8247E
:106A4000F76AF736670FF66E6A0EF722000EF86ED9
:106A5000FB6E0A00F550FA6E0800F55021BCF28C6E
:106A600021BEF28EF96E086A0C6A106A146A186AFE
:106A7000206A206A1C6A0701465105081BE144513F
:106A8000442B036A1C0FE96E060E0320EA6EEFCF5B
:106A900001F001C026F909012651310804E1000185
:106AA000738F06D009012651300803E10001A5DFEC
:106AB000090107014651040822E191A40FD0310ECB
:106AC00009013B6F07014351432B036AAC0FE96E89
:106AD000060E0320EA6E3BC9EFFF0ED0300E09010F
:106AE0003B6F07014351432B036AAC0FE96E060E5F
:106AF0000320EA6E3BC9EFFF0001A5DD070100019D
:106B00004EEF45F007014651050819E1010E090154
:106B1000286F000127DD01C026F9080E09012A6F40
:106B200026C92BF90001EAEC23F009013F6B090E9D
:106B30003E6F44C040F9000111EC12F007014651CC
:106B4000040813E109012A6B2B6B0001EAEC23F026
:106B500001C026F909012B6B26C92AF9010E2C6FF9
:106B60002D6B000135DD6FDD0701000158EF45F0A9
:106B7000875331E141AA2FD00901296B29510F0810
:106B800015E3036A2951550FE96E000E0320EA6EE2
:106B9000EF50200B09E1036A2951550FE96E000EF1
:106BA0000320EA6EFF0EEF6E292BE8D741A201D039
:106BB000288D2C6AF2BC2C8CF29CF2BE2C8EF29E9C
:106BC00028C961F900010CEC0EF02CBCF28C2CBE33
:106BD000F28E015002D0000E016E000C07014651EA
:106BE0000608D8A407D1020E0901286F0001BADCFB
:106BF00002C027F901C026F9090126C900F0275172
:106C0000036E04E10052000151E00901035005E167
:106C1000010E005C000159E00901035006E1020E7B
:106C2000005C0001D8B460D00901035006E1030EF6
:106C3000005C0001D8B465D00901035006E1040EE0
:106C4000005C0001D8B46CD00901035006E1050EC8
:106C5000005C0001D8B473D00901035006E1060EB0
:106C6000005C0001D8B47AD00901035006E1070E98
:106C7000005C0001D8B481D00901035006E1080E80
:106C8000005C0001D8B488D00901035006E1090E68
:106C9000005C0001D8B48FD00901035006E10A0E50
:106CA000005C0001D8B496D00901A3D0010E0901FF
:106CB000286F00015DDF015206E1010E0901286F16
:106CC0000001B4EC2AF0090194D0020E0901286FEA
:106CD00000014EDF015206E1020E0901286F00019A
:106CE000B4EC2AF0090185D00901286B000140DFCE
:106CF000015205E10901286B0001B4EC2AF00901F9
:106D000078D0030E0901286F000132DF015206E13D
:106D1000030E0901286F0001B4EC2AF0090169D0C3
:106D2000040E0901286F000123DF015206E1040E61
:106D30000901286F0001B4EC2AF009015AD0050EB0
:106D40000901286F000114DF015206E1050E090157
:106D5000286F0001B4EC2AF009014BD0060E09019E
:106D6000286F000105DF015206E1060E0901286FB8
:106D70000001B4EC2AF009013CD0070E0901286F8C
:106D80000001F6DE015206E1070E0901286F00013D
:106D9000B4EC2AF009012DD0080E0901286F00017A
:106DA000E7DE015206E1080E0901286F0001B4EC8C
:106DB0002AF009011ED0090E0901286F0001D8DE52
:106DC000015206E1090E0901286F0001B4EC2AF016
:106DD00009010FD00A0E0901286F0001C9DE015216
:106DE00006E10A0E0901286F0001B4EC2AF009013E
:106DF00000D00701465104081AE1036A00018651D8
:106E0000130FE96E090E0320EA6EEF50036A0901C1
:106E1000266F03C027F927C92BF926C92AF9020EC4
:106E20002C6F2D6B0001E8EC32F00DDC0701000146
:106E300060EF45F007014451442B036A1C0FE96ED3
:106E4000060E0320EA6EEFCF01F001C027F9090119
:106E50000150600806E227517A0803E32751DF0B4F
:106E600001D02751266F2651500A000103E0080A7D
:106E70004FE09CD00701465106081FE14451442BC6
:106E8000036A1C0FE96E060E0320EA6EEFCF01F0D5
:106E900001C026F9300E0901265D276F080E2A6F02
:106EA00027C92BF9000148EC1DF0030E09012A6FD8
:106EB0002B6B000148EC1DF007014651050826E147
:106EC00026C93BF94351432B036AAC0FE96E060E0A
:106ED0000320EA6E3BC9EFFF09012A6B2B6B00010F
:106EE00048EC1DF0300E01240901266F26C93BF93C
:106EF00007014351432B036AAC0FE96E060E0320D2
:106F0000EA6E3BC9EFFF000123EC33F000014ED0E5
:106F10000701465106081FE14451442B036A1C0F28
:106F2000E96E060E0320EA6EEFCF01F001C026F9EC
:106F3000300E0901265D276F080E2A6F27C92BF92D
:106F4000000134EC1CF0030E09012A6F2B6B0001C9
:106F500034EC1CF007014651050826E126C93BF92F
:106F60004351432B036AAC0FE96E060E0320EA6E11
:106F70003BC9EFFF09012A6B2B6B000134EC1CF0BD
:106F8000300E01240901266F26C93BF90701435140
:106F9000432B036AAC0FE96E060E0320EA6E3BC971
:106FA000EFFF000123EC33F0000100D068EF45F063
:106FB00007014451442B036A1C0FE96E060E03209F
:106FC000EA6EEFCF01F001C028F909010150600815
:106FD00006E228517A0803E32851DF0B01D028513B
:106FE000276F27514F0844E10701465106081AE16F
:106FF000010E0901286F0001B2EC32F001C026F940
:10700000080E09012A6F26C92BF900014DEC19F071
:1070100009013F6B090E3E6F44C040F9000111ECBD
:1070200012F007014651050822E109012A6B2B6B7A
:1070300000014DEC19F001C026F927C93BF9070101
:107040004351432B036AAC0FE96E060E0320EA6E30
:107050003BC9EFFF09012B6B26C92AF9010E2C6FE2
:107060002D6B0001E8EC32F023EC33F0070109014D
:10707000000172EF45F009012E6B07014451442BCA
:10708000036A1C0FE96E060E0320EA6EEFCF01F0D3
:1070900001C030F909010150600806E230517A0858
:1070A00003E33051DF0B01D030512F6F2F513908DE
:1070B00002E2070E2F5F2F510F0B006E00382E6F6C
:1070C000F00E2E1707014451442B036A1C0FE96E82
:1070D000060E0320EA6EEFCF01F001C030F909017E
:1070E0000150600806E230517A0803E33051DF0BAB
:1070F00001D030512F6F2F51390802E2070E2F5F58
:107100002F510F0B2E132E510701452709012EC9B0
:1071100001F00001000C09012D39006E0F0E001660
:10712000005030092E6F2E51390802E2070E2E272B
:107130002EC93BF907014351432B036AAC0FE96E9B
:10714000060E0320EA6E3BC9EFFF09012D510F0B1C
:1071500030092E6F2E51390802E2070E2E272EC954
:107160003BF907014351432B036AAC0FE96E060E4E
:107170000320EA6E3BC9EFFF09012D5107014227A9
:107180000001000C09012E6B2E513F0830E32D51F8
:10719000030822E3036A2E51540FE96E010E032007
:1071A000EA6E2D51036E2C512C2BD8B42D2B316F40
:1071B00003C032F9F2CF33F9F29CF29E32C9AAFF32
:1071C00031C9A9FFA69CA69EA680A85033BDF28C0B
:1071D00033BFF28EEF6E09D0036A2E51540FE96E61
:1071E000010E0320EA6EFF0EEF6E2E2BCDD70001AD
:1071F00043EF39F00701456B00013DDF01C027F97E
:107200003ADF01C028F937DF01C029F934DF07016F
:10721000426B030E436F27C92DF900017CDF28C99B
:107220002DF979DF070146510C0852E1455350E131
:10723000090127510308D8B002D0070149D02951CC
:107240004008D8B002D0070143D02B6B27C92AF9D8
:107250002AC92DF92C6B28512C252A6F000E2D21BF
:107260002B6F29512A252C6F000E2B212D6F04081E
:107270002EE303E12C5100082AE32BC92DF92AC97A
:107280002CF900017FD729C92DF945DF0901266BAB
:107290002951265D10E2036A2651540FE96E010E52
:1072A0000320EA6EEFCF2CF92CC92DF9000133DF52
:1072B0000901262BEDD70701421D09012C6F2C2B4C
:1072C0002CC92DF9000127DF23EC33F00901070158
:1072D00000017CEF45F009012F6B2E512F5D34E248
:1072E0002D51030831E32D51036E2C512C2BD8B4B2
:1072F0002D2B306F03C031F9036A2F51540FE96E03
:10730000010E0320EA6EEFCF32F931C949F930C9D5
:1073100048F932C94AF949C9AAFF48C9A9FF4AC967
:10732000A8FFA69CA69EA684F2CF4BF9F29CF29EE3
:10733000550EA76EAA0EA76EA6824B51F212A6B2E8
:10734000FED7A6922F2BC9D7000110EF3AF0070104
:10735000456B000190DE01C027F98DDE01C028F9E0
:107360008ADE01C029F909012B6B27C92AF92AC92C
:107370002DF92C6B2C5128112A6F2DC92BF90701DF
:10738000426B030E436F27C92DF90001C4DE28C9E3
:107390002DF9C1DE070146518C080BE3D890090195
:1073A00029350C0F0701465D04E14651010B010828
:1073B00001E146D009012951400841E329512A251C
:1073C0002C6F000E2B212D6F2D5339E12C51F0081D
:1073D00036E3266B2951265D15E2036A2651540FC8
:1073E000016E010E032201C02CF903C02DF900012A
:1073F00042DE2DC9EAFF2CC9E9FF01C0EFFF0901F8
:10740000262BE8D7000137DE0701455301E018D0ED
:107410002BC92DF92AC92CF929C92EF900015BD7EE
:1074200029C92DF978DE0701421D09012C6F2C2B8B
:107430002CC92DF900016FDE23EC33F0090107019F
:10744000000184EF45F0010E0901286F276B2851D8
:10745000030825E303E12751FE0821E328C949F980
:1074600027C948F9FF0E4A6F49C9AAFF48C9A9FFB1
:107470004AC9A8FFA69CA69EA684F2CF4BF9F29C0F
:10748000F29E550EA76EAA0EA76EA6824B51F2125F
:10749000A6B2FED7A692272BD8B4282BD8D70001A6
:1074A000E3EF3AF007014451442B036A1C0FE96EE5
:1074B000060E0320EA6EEFCF01F001C027F90901A3
:1074C0000150600806E227517A0803E32751DF0BD9
:1074D00001D02751266F26515408D8A475D0070132
:1074E00046510908D8B402D009016ED04451442B4A
:1074F000036A1C0FE96E060E0320EA6EEFCF01F05F
:1075000001C027F909010150600806E227517A08F5
:1075100003E32751DF0B01D02751360801E054D097
:1075200007014451442B036A1C0FE96E060E032029
:10753000EA6EEFCF01F001C027F9090101506008A0
:1075400006E227517A0803E32751DF0B01D02751C8
:10755000380801E039D007014451442B036A1C0F5D
:10756000E96E060E0320EA6EEFCF01F001C027F9A5
:1075700009010150600806E227517A0803E3275108
:10758000DF0B01D02751320801E01ED00701445122
:10759000442B036A1C0FE96E060E0320EA6EEFCF40
:1075A00001F001C027F909010150600806E22751E6
:1075B0007A0803E32751DF0B01D02751310801E09E
:1075C00003D0000140D7090100018CEF45F007010D
:1075D0004651050818E1010E0901286F0001B2ECBF
:1075E00032F001C026F9080E09012A6F26C92BF9CD
:1075F00000012BEC1FF0030E09012A6F2B6B000119
:107600002BEC1FF007014651040815E109012A6B14
:107610002B6B00012BEC1FF001C026F909012B6B2D
:1076200026C92AF9020E2C6F2D6B0001E8EC32F00E
:1076300023EC33F00701000196EF45F0020E6C5D7C
:10764000F50F23E20B0F57EF3BF06F99796B786BD7
:107650001CD06F9F7F6B7E6B18D06F91756B746BB6
:1076600014D06F9312D06F95776B766B0ED06F9BA3
:107670000CD06F9D7B6B7A6B08D0709106D07093A5
:1076800004D070957D6B7C6B00D06C6B6F5170116A
:107690000DE18E8E8A949EEC22F0736BFDEC34F03B
:1076A000726B716B210E486EF5C888F0000CF2CF3A
:1076B00021F0F29CF29EE824F76AF736DF0FF66EAF
:1076C000760EF722000EF86EFB6E0A00F550FA6E89
:1076D0000800F55021BCF28C21BEF28EF96E5A766C
:1076E000627666768A764A766E76727652767A76A2
:1076F0007E7682760701465105081DE14451442BF0
:10770000036A1C0FE96E060E0320EA6EEFCF01F04C
:1077100001C026F909010150600806E226517A08E5
:1077200003E32651DF0B01D02651430803E100019A
:1077300085DF09010701465104080DE109012B6BA2
:107740006CC02AF9020E2C6F2D6B0001E8EC32F0B0
:1077500023EC33F0070100019EEF45F00901326B85
:107760008A0E316F336B070E346F0001C7EC17F0D0
:107770006A6B6AC069F069C068F068C067F0E4ECE1
:1077800017F0B76A696A6A6A736A706A09013F6BBF
:107790000A0E3E6F88C040F9000111EC12F0000C97
:1077A00009012851FE0804E14A5202E1FE0E4A6E28
:1077B000AAC029F94A50FE0A000115E0010A18E0A2
:1077C000FF0A1CE0010A25E0030A45E0010AD8B4DB
:1077D00064D0070AD8B484D0010AD8B4A4D0030A6C
:1077E000D8B4C4D0CFD0908090829094908609D1A4
:1077F0000901116B106B4A6A0001C4D009012951BB
:10780000320805E2010E4A6E116F770E106F00010B
:10781000B9D0090129512F0813E311C903F0105100
:10782000D8B4110710072A6F03C02BF92A5307E1B8
:107830002B5305E14A6A010E116F770E106F09D0C4
:107840002951360806E2020E4A6E010E116F770EBC
:10785000106F000197D009012951340813E311C9B1
:1078600003F01051D8B4110710072A6F03C02BF989
:107870002A5307E12B5305E1010E4A6E116F770E73
:10788000106F09D029513B0806E2030E4A6E010E23
:10789000116F770E106F000175D009012951390859
:1078A00014E311C903F01051D8B4110710072A6F5F
:1078B00003C02BF92A5308E12B5306E1020E4A6E4E
:1078C000010E116F770E106F09D02951400806E2A2
:1078D000040E4A6E010E116F770E106F000152D028
:1078E000090129513E0814E311C903F01051D8B41D
:1078F000110710072A6F03C02BF92A5308E12B53F5
:1079000006E1030E4A6E010E116F770E106F09D05B
:107910002951450806E2050E4A6E010E116F770ED9
:10792000106F00012FD009012951430814E311C938
:1079300003F01051D8B4110710072A6F03C02BF9B8
:107940002A5308E12B5306E1040E4A6E010E116F13
:10795000770E106F09D029514F0806E2060E4A6EC5
:10796000010E116F770E106F00010CD00901295123
:107970004D0806E3050E4A6E010E116F770E106F6B
:10798000000100D009012A6B2B6B00012BEC1FF0CA
:1079900001C029F9090129514A5C02E229C94AF0CA
:1079A0004A50F90F2FE2070F000104EF3DF09090CD
:1079B000909290949096090125D090809082908426
:1079C000909609011FD09080908290949086090132
:1079D00019D09080908290949096090113D0908055
:1079E00090929084908609010DD09080909290940E
:1079F0009086090107D0908090929094909609010A
:107A000001D009010001000CF2CF21F0F29CF29E9E
:107A1000E824F76AF736390FF66E7A0EF722000E71
:107A2000F86EFB6E0A00F550FA6E0800F55021BCA6
:107A3000F28C21BEF28EF96EAE79BA79C679D2791E
:107A4000DE79EA79F67907014451442B036A1C0F69
:107A5000E96E060E0320EA6EEFCF01F001C027F9B0
:107A600009010150600806E227517A0803E3275113
:107A7000DF0B01D02751266F2651530849E107013A
:107A800046510508D8B402D0090142D02C6AF2BC94
:107A90002C8CF29CF2BE2C8EF29E000132EC0EF089
:107AA0002CBCF28C2CBEF28E919609012E6B00013B
:107AB00045EC24F02C6AF2BC2C8CF29CF2BE2C8E8D
:107AC000F29E320E0901616F00010CEC0EF02CBC2D
:107AD000F28C2CBEF28E42DEFE0E0901286F0001F0
:107AE0005FDEC80E0901286F00011FEC10F09096B0
:107AF00090949082908084AC02D0535207E0010EA3
:107B00000901286F00011FEC10F0F5D7FF000901F3
:107B10000001A6EF45F00901266B07014651040854
:107B200011E14A5202E04AC026F909012B6B26C92D
:107B30002AF9020E2C6F2D6B0001E8EC32F023ECD9
:107B400033F007010001AEEF45F007014451442B2B
:107B5000036A1C0FE96E060E0320EA6EEFCF01F0F8
:107B600001C027F909010150600806E227517A088F
:107B700003E32751DF0B01D02751266F26514D0813
:107B800026E1070146510508D8B402D009011FD0EB
:107B9000400E486E41A20FD02C6AF2BC2C8CF29C95
:107BA000F2BE2C8EF29E000132EC0EF02CBCF28C58
:107BB0002CBEF28E0701919C8B9209013F6B070E40
:107BC0003E6F86C040F9000111EC12F0090100017E
:107BD000B8EF45F009012A51010A000111E0030A3A
:107BE00010E0010A0FE0040A0EE0030A0DE0010AAA
:107BF0000DE0030A0DE00E0A31E0080A39E038D042
:107C000038D037D036D035D0448E33D0449E31D0A2
:107C100044BE12D009012C6B2C510001C3EC0AF0B8
:107C2000000909E009012C2B326F0001EAEC16F083
:107C30000901F2D7000111D009012C6B2C51000170
:107C4000DAEC0AF0000909E009012C2B326F00017F
:107C5000EAEC16F00901F2D700010BD009012B5311
:107C600002E1449E03D02B2D01D0448E000101D0AF
:107C700000D044AE02D0010E01D0000E016E000C07
:107C800007014651050821E14451442B036A1C0FAA
:107C9000E96E060E0320EA6EEFCF01F0300E015CB4
:107CA0000901266F2651010807E3080E2A6F26C92D
:107CB0002BF900018FDF09013F6B090E3E6F44C0B5
:107CC00040F9000111EC12F00701465104081CE1D3
:107CD00009012A6B2B6B00017DDF01C026F9300EF4
:107CE00009012625276F27C93BF907014351432B7B
:107CF000036AAC0FE96E060E0320EA6E3BC9EFFF84
:107D0000000123EC33F007010001C2EF45F0310E12
:107D10000901266F0701465105082FE14451442B04
:107D2000036A1C0FE96E060E0320EA6EEFCF01F026
:107D30000150300822E1400E486E41A20FD02C6A5B
:107D4000F2BC2C8CF29CF2BE2C8EF29E000132EC26
:107D50000EF02CBCF28C2CBEF28E0701919C8B9203
:107D600009013F6B070E3E6F86C040F9000111EC20
:107D700012F0300E0901266F07014651040810E188
:107D800026C93BF94351432B036AAC0FE96E060E3B
:107D90000320EA6E3BC9EFFF000123EC33F007013B
:107DA0000001CCEF45F041B211D047520FE188A05D
:107DB00003D0260E476E0AD06F51701107E16A9FFB
:107DC0006A8D8A8A8A88418229EC0EF0000C8753DA
:107DD00038E141AA36D00901276B27510F081BE370
:107DE000036A2751550FE96E000E0320EA6EEF502B
:107DF0003F0B286F2851340803E02851330809E16C
:107E0000036A2751550FE96E000E0320EA6EFF0E3C
:107E1000EF6E272BE2D72C6AF2BC2C8CF29CF2BEC0
:107E20002C8EF29E740E616F00010CEC0EF02CBCD7
:107E3000F28C2CBEF28E015202E1B5DF01D0428AF3
:107E400001D0B1DF000C07014651050827E144517C
:107E5000442B036A1C0FE96E060E0320EA6EEFCF77
:107E600001F001C026F909012651310804E10001A1
:107E7000AEDF12D00901265130080FE12C6AF2BCA6
:107E80002C8CF29CF2BE2C8EF29E000139EC0EF08E
:107E90002CBCF28C2CBEF28E09010701465104085D
:107EA00023E141A20FD0310E09013B6F070143517D
:107EB000432B036AAC0FE96E060E0320EA6E3BC942
:107EC000EFFF0ED0300E09013B6F07014351432BEA
:107ED000036AAC0FE96E060E0320EA6E3BC9EFFFA2
:107EE000000123EC33F007010001D4EF45F0070156
:107EF000465107082CE1030E0901286F0001B2EC7E
:107F000032F002C027F901C026F90901275303E125
:107F100026514F081BE2275319E12651780816E332
:107F2000500E265F000E275B26C928F9296B080E24
:107F30002A6F26C92BF9000133EC1AF0030E090150
:107F40002A6F2B6B000133EC1AF00901070146512F
:107F500004081DE1090E09012A6F2B6B000133ECA7
:107F60001AF00901276B01C026F9500E2625286F4B
:107F7000000E2721296F2B6F28C92AF9030E2C6FB9
:107F80002D6B0001E8EC32F023EC33F00701000127
:107F9000DEEF45F007014651050822E14451442B2C
:107FA000036A1C0FE96E060E0320EA6EEFCF01F0A4
:107FB000300E015C0901266F2651010808E3080E06
:107FC0002A6F26C92BF90001DBEC24F009013F6B75
:107FD000090E3E6F44C040F9000111EC12F0070198
:107FE000465104081DE109012A6B2B6B0001DBECF3
:107FF00024F001C026F9300E09012625276F27C974
:108000003BF907014351432B036AAC0FE96E060E9F
:108010000320EA6E3BC9EFFF000123EC33F00701B8
:108020000001E6EF45F00901386BF00E376F0001F3
:1080300032EC13F002C036F901C035F909013551AF
:10804000470803E1362D01D020D03E6BF00E3D6F86
:10805000010E406F470E3F6F0001BCEC11F00901AB
:10806000386BF00E376F000132EC13F002C036F9B6
:1080700001C035F9050E0901376F36C939F935C91F
:1080800038F9000145EC12F009012A51F80F57E2C6
:10809000080F0001A5EF40F0090151D009014FD0B0
:1080A00009014DD009014BD0090149D0090147D040
:1080B000090145D0200E09012B6F460E2C6F500E82
:1080C0002D6F200E2E6F3639376F0F0E3717375141
:1080D0000F0B396F3A6B300E39252F6F36510F0B5E
:1080E000396F3A6B300E3925306F2E0E316F3631C5
:1080F000386F3531376F38333733383337333833B8
:1081000037330F0E381737510F0B396F3A6B300E6C
:108110003925326F35510F0B376F386B300E3725DD
:10812000336F346B090E3D6F2B0E3C6F3E6B090EA7
:108130003F6F0001F8EC15F0090101D0090135C9C4
:1081400001F036C902F00001000CF2CF21F0F29CE0
:10815000F29EE824F76AF7367B0FF66E810EF7225F
:10816000000EF86EFB6E0A00F550FA6E0800F5502E
:1081700021BCF28C21BEF28EF96E98809C80A0808A
:10818000A480A880AC80B480B08007014451442B07
:10819000036A1C0FE96E060E0320EA6EEFCF01F0B2
:1081A00001C029F909010150600806E229517A0845
:1081B00003E32951DF0B01D02951266F26514D08C9
:1081C00041E1070146510508D8B402D009013AD06F
:1081D00026C93BF94351432B036AAC0FE96E060EE7
:1081E0000320EA6E3BC9EFFF09012A6B00011BDF88
:1081F00002C028F901C027F928C929F909012A6B09
:1082000028C92BF92C6B28C92DF900018BEC38F00B
:108210002E0E09013B6F07014351432B036AAC0F3C
:10822000E96E060E0320EA6E3BC9EFFF090127C97C
:1082300029F92A6B27C92DF900018BEC38F023ECC2
:1082400033F009010001F0EF45F007014451442BE0
:10825000036A1C0FE96E060E0320EA6EEFCF01F0F1
:1082600001C027F909010150600806E227517A0888
:1082700003E32751DF0B01D02751266F26514D080C
:108280002EE1070146510508D8B402D0090127D0D4
:10829000000129EC18F033EC25F0CAEC25F09EEC37
:1082A00011F009013E6B090E3D6F030E3F6F000197
:1082B00058EC11F001C044F02C6AF2BC2C8CF29CFA
:1082C000F2BE2C8EF29E39EC0EF02CBCF28C2CBE41
:1082D000F28E0E0E896FA56B7D0EA46F0901000151
:1082E000F8EF45F007014651040817E109012A6B30
:1082F00000011BEC26F002C027F901C026F927C9AE
:108300002BF926C92AF9050E09012C6F2D6B0001E6
:10831000E8EC32F023EC33F00701000102EF46F005
:1083200007014651050822E14451442B036A1C0F02
:10833000E96E060E0320EA6EEFCF01F0300E015C0D
:108340000901266F2651010808E3080E2A6F26C985
:108350002BF90001A4EC1FF009013F6B090E3E6FE1
:1083600044C040F9000111EC12F007014651040825
:108370001DE109012A6B2B6B0001A4EC1FF001C069
:1083800026F9300E09012625276F27C93BF9070179
:108390004351432B036AAC0FE96E060E0320EA6ECD
:1083A0003BC9EFFF000123EC33F0070100010AEFA6
:1083B00046F00701465104080EE1ABC02BF9AAC0F4
:1083C0002AF9030E09012C6F2D6B0001E8EC32F045
:1083D00023EC33F00701000114EF46F0070146518A
:1083E00006081FE1020E0901286F0001B2EC32F00D
:1083F00001C026F9080E09012A6F26C92BF90001D0
:10840000CBEC1EF0030E09012A6F2B6B0001CBECA5
:108410001EF0070E09012A6F2B6B0001CBEC1EF03A
:1084200007014651040815E109012A6B2B6B000175
:10843000CBEC1EF001C026F909012B6B26C92AF9E5
:10844000020E2C6F2D6B0001E8EC32F023EC33F0C0
:10845000070100011CEF46F007014451442B036A59
:108460001C0FE96E060E0320EA6EEFCF01F001C08B
:1084700028F909010150600806E228517A0803E34F
:108480002851DF0B01D02851276F27515408D8A459
:10849000CCD0070146510608D8A4AAD0010E090184
:1084A000286F0001B2EC32F001C026F94850F00B01
:1084B000200A03E0700A05E09AD048C01EF988C07F
:1084C0001FF909012651FC0FD8B08FD0040F00010D
:1084D00018EF43F02C6AF2BC2C8CF29CF2BE2C8E6E
:1084E000F29E32EC0EF02CBCF28C2CBEF28E9196E9
:1084F00009012E6B000145EC24F02C6AF2BC2C8C97
:10850000F29CF2BE2C8EF29E320E0901616F0001C8
:108510000CEC0EF02CBCF28C2CBEF28EAEEC3BF0D0
:10852000FE0E0901286F0001D0EC3BF0C80E0901D6
:10853000286F00011FEC10F090969094908290802C
:1085400009013F6BFD0E3E6FFF0E406F000111EC05
:1085500012F084AC02D0535207E0010E0901286FDB
:1085600000011FEC10F0F5D7FF001EC948F01FC92D
:1085700088F009013AD02C6AF2BC2C8CF29CF2BE35
:108580002C8EF29E39EC0EF02CBCF28C2CBEF28EAE
:10859000510E486E090E886F090127D02C6AF2BC73
:1085A0002C8CF29CF2BE2C8EF29E39EC0EF02CBC80
:1085B000F28C2CBEF28E520E486E090E886F0901A5
:1085C00014D02C6AF2BC2C8CF29CF2BE2C8EF29E43
:1085D00039EC0EF02CBCF28C2CBEF28E530E486E91
:1085E000090E886F090101D009018E8E0001070173
:1085F0004651050819E127C93BF94351432B036A4A
:10860000AC0FE96E060E0320EA6E3BC9EFFF0901CD
:108610002B6B26C92AF9010E2C6F2D6B0001E8EC9B
:1086200032F023EC33F007010901000123EF46F09B
:10863000F2CF21F0F29CF29EE824F76AF736610F40
:10864000F66E860EF722000EF86EFB6E0A00F550ED
:10865000FA6E0800F55021BCF28C21BEF28EF96E44
:10866000D48476859C85C28507014651050804E0BF
:1086700046510608D8A478D04451442B036A1C0FF5
:10868000E96E060E0320EA6EEFCF01F0300E015CBA
:108690000901266F2651FC0F66E2040F000104EF6A
:1086A00044F0080E09012D6F26C92EF9000114ECC3
:1086B0001EF0030E09012D6F2E6B000114EC1EF04D
:1086C000090151D0080E09012D6F26C92EF90001AC
:1086D00014EC1EF0030E09012D6F2E6B000114EC3B
:1086E0001EF0090140D0080E09012D6F26C92EF990
:1086F000000114EC1EF0030E09012D6F2E6B00011A
:1087000014EC1EF00701465106082AE14451442B9F
:10871000036A1C0FE96E060E0320EA6EEFCF01F02C
:10872000300E015C0901266F2651010819E3080E7D
:108730002A6F26C92BF9000150EC24F0070E09011D
:108740002A6F26C92BF9000150EC24F009013F6B78
:10875000090E3E6F44C040F9000111EC12F009010E
:10876000090101D009010701465104084AE1090144
:108770002D6B2E6B000114EC1EF001C026F9300E9B
:1087800009012625276F27C93BF907014351432BD0
:10879000036AAC0FE96E060E0320EA6E3BC9EFFFD9
:1087A000090126530FE1310E3B6F07014351432B63
:1087B000036AAC0FE96E060E0320EA6E3BC9EFFFB9
:1087C0001CD009012651030818E12A6B2B6B00010C
:1087D00050EC24F001C026F9300E09012625276F40
:1087E00027C93BF907014351432B036AAC0FE96EDC
:1087F000060E0320EA6E3BC9EFFF000123EC33F0C5
:10880000070100012CEF46F0F2CF21F0F29CF29E1E
:10881000E824F76AF736390FF66E880EF722000E55
:10882000F86EFB6E0A00F550FA6E0800F55021BC98
:10883000F28C21BEF28EF96EA286C486C486E686CC
:108840000701465104084EE1B3C03EF9B2C03DF9FC
:108850000901406B0A0E3F6F0001ABEC11F00901FA
:108860000230276F0130266F273326332733263314
:108870002733263327332633070E271727C92BF92B
:1088800026C92AF9030E2C6F2D6B0001E8EC32F09B
:10889000200E09013B6F07014351432B036AAC0FC4
:1088A000E96E060E0320EA6E3BC9EFFFB1C03EF948
:1088B000B0C03DF90901406B0A0E3F6F0001ABECFF
:1088C00011F002C026F90901276B27C92BF926C927
:1088D0002AF9030E2C6F2D6B0001E8EC32F023EC2B
:1088E00033F00701000135EF46F00901266B276BD5
:1088F00007014651040831E14CC12BF94BC12AF95B
:10890000030E09012C6F2D6B0001E8EC32F0200EF4
:1089100009013B6F07014351432B036AAC0FE96E1A
:10892000060E0320EA6E3BC9EFFF01014A5303E143
:108930004951090804E24AC127F949C126F927C962
:108940002BF926C92AF9030E09012C6F2D6B0001A2
:10895000E8EC32F023EC33F0070100013EEF46F083
:108960000701446B436B4451442B036A1C0FE96EAF
:10897000060E0320EA6EEFCF01F001C023F90901D2
:1089800023513B0807E13B0E266F00019FEF32F0B9
:1089900078D1090123515E08D8A474D15E0E3B6FD3
:1089A00007014351432B036AAC0FE96E060E032007
:1089B000EA6E3BC9EFFF4451442B036A1C0FE96E7A
:1089C000060E0320EA6EEFCF01F001C026F909017F
:1089D0002651600806E226517A0803E32651DF0B90
:1089E00001D02651246F24C93BF907014351432B81
:1089F000036AAC0FE96E060E0320EA6E3BC9EFFF77
:108A00004451442B036A1C0FE96E060E0320EA6EE4
:108A1000EFCF01F001C026F909012651600806E2F6
:108A200026517A0803E32651DF0B01D02651256F2A
:108A300025C93BF907014351432B036AAC0FE96E8B
:108A4000060E0320EA6E3BC9EFFF410E0901245DCB
:108A5000E80FD8B017D1180F000145EF46F0090113
:108A60002551490805E1000170EF33F00AD10901F1
:108A700025514C0805E1000193EF33F002D10901C3
:108A80002551520805E10001D8EF33F0FAD0090171
:108A90002551540804E100013BEF35F0F2D000010C
:108AA000F0D009012551430805E1000182EF35F0BE
:108AB000E8D0090125514E0805E10001EEEF35F03F
:108AC000E0D009012551520804E100011AEF37F006
:108AD000D8D00001D6D0090125514D0804E100018C
:108AE000D8EF37F0CED00001CCD009012551520883
:108AF00005E10001FAEF38F0C4D00901255157080B
:108B000005E10001A7EF39F0BCD009012551460865
:108B100004E1000152EF3AF0B4D00001B2D00901F3
:108B20002551430805E10001E7EF3AF0AAD0090119
:108B300025514C0805E100017AEF3BF0A2D0090174
:108B40002551520805E1000123EF3DF09AD00901BB
:108B50002551530804E100018BEF3DF092D0000154
:108B600090D009012551440804E10001A5EF3DF032
:108B700088D0000186D009012551480804E1000190
:108B800040EF3EF07ED000017CD0090125514E0817
:108B900005E1000187EF3EF074D00901255153082B
:108BA00004E1000123EF3FF06CD000016AD009011D
:108BB00025514A0805E1000177EF3FF062D0090135
:108BC00025514F0804E10001CAEF3FF05AD00001DF
:108BD00058D009012551560805E10001C5EF40F0C4
:108BE00050D009012551500804E1000125EF41F062
:108BF00048D0000146D0090125514E0805E1000189
:108C000072EF41F03ED009012551500804E1000106
:108C100090EF41F036D0000134D0090125514D08C4
:108C200005E10001D9EF41F02CD00901255152088E
:108C300005E10001EEEF41F024D009012551530870
:108C400003E1000109D41DD000011BD00901255109
:108C5000490803E1000108D514D0000112D0090130
:108C60002551490803E10001EBD50BD0000109D0E3
:108C700009012551530803E1000137D602D0000154
:108C800000D009010001ABEF46F0F2CF21F0F29CD9
:108C9000F29EE824F76AF736BB0FF66E8C0EF722C9
:108CA000000EF86EFB6E0A00F550FA6E0800F550E3
:108CB00021BCF28C21BEF28EF96E5E8AA28A828C71
:108CC000D68AEA8A1E8B828C828C828C828C828CE1
:108CD000628B828C768B8A8BAE8B828CD28BF68B5E
:108CE0001A8C828C5E8C708C4C8C07013C5100017C
:108CF00003E0010A08E000D006011C6B0701466B87
:108D0000010E3C6F0001070140513F5D2EE04051D4
:108D1000402B1C0FE96E050EEA6ED8B0EA2AEFCFA1
:108D200022F9090107014651462B036A1C0FE96E1F
:108D3000060E0320EA6E22C9EFFF036A46511C0F9C
:108D4000E96E060E0320EA6EEF6A090122513B0824
:108D500005E1000105D607013C6B08D0070146512B
:108D60008E0802E23C6B02D0CFD700D000013DEF6D
:108D700064F0010E04011825175D0AE0940E182511
:108D8000E96E010EEA6ED8B0EA2A24C9EFFF182B6B
:108D90009D880001E1EF48F00901276B27510A087F
:108DA0001EE3036A27512A0F016E090E03220150A8
:108DB000366F03C037F904011551152B036A940F60
:108DC000E96E030E0320EA6EEFCF01F037C9EAFF28
:108DD00036C9E9FF01C0EFFF0901272BDFD72A5170
:108DE000300806E12B51300803E12C51300803E034
:108DF0000F0E016E9CD0300E2D5D376F3E6B3D6FB8
:108E0000406B640E3F6F0001ABEC11F002C039F90A
:108E100001C038F9300E09012E5D3B6F3E6B3D6F8E
:108E2000406B0A0E3F6F0001ABEC11F001500901DD
:108E300038253C6F025039213D6F2F513C253E6F44
:108E4000000E3D213F6F300E3E5D286F000E3F59F2
:108E5000296F295332E1285172082FE3295318E171
:108E600028512D0815E3295306E128510F0803E383
:108E70000F0E016E5CD0295307E12851180804E356
:108E8000010E016E54D003D0020E016E50D014D0EA
:108E9000295306E128513D0803E3000E016E47D037
:108EA000295307E12851540804E3030E016E3FD013
:108EB00003D0040E016E3BD038D0295318E128515D
:108EC000E50815E3295306E12851A10803E3050E3F
:108ED000016E2DD0295307E12851C20804E3060E84
:108EE000016E25D003D0070E016E21D01ED029516E
:108EF000010807E303E12851030803E3080E016EAC
:108F000016D02951010807E303E12851490803E37A
:108F1000090E016E0CD02951020807E303E1285124
:108F20002F0803E30A0E016E02D00F0E016E00013E
:108F3000000C0901269126830401156B1551152B90
:108F4000036A940FE96E030E0320EA6EEFCF01F07F
:108F500001C027F909010150600806E227517A088B
:108F600003E32751DF0B01D02751236F0401155173
:108F7000152B036A940FE96E030E0320EA6EEFCF00
:108F800001F001C027F909010150600806E22751EC
:108F90007A0803E32751DF0B01D02751246F2351B7
:108FA00046084EE12451410A000107E0030A10E09F
:108FB000100A19E0060A2CE040D0EEDE01C025F9C7
:108FC000090125510F0801E1E3D025C94FF137D040
:108FD000E3DE01C025F9090125510F0801E1D8D0D0
:108FE00025C950F12CD004011551152B036A940F9B
:108FF000E96E030E0320EA6EEFCF01F00150030B80
:109000000901256F2551020802E325C952F117D045
:1090100004011551152B036A940FE96E030E03200A
:10902000EA6EEFCF01F00150030B0901256F2551C6
:10903000020802E325C953F102D00901A9D070D07A
:1090400023514908D8A46BD024514608D8A467D02E
:109050000001A2DE01C025F9090125510F0801E137
:1090600097D0300E0301B05D09012693E8B0268346
:109070000301B451010B09012691E8B026810301D7
:10908000B251300A000105E0010A1FE0030A3BE08B
:1090900041D025C94FF1090126A30CD00101536B22
:1090A000090126A102D0010E01D0000E0101526F6C
:1090B0000BD009010101526B090126A102D0010E5A
:1090C00001D0000E0101536F28D025C950F10901CC
:1090D00026A30DD0010E0101536F090126A102D074
:1090E000000E01D0010E0101526F0CD00901010EDA
:1090F0000101526F090126A102D0000E01D0010E1C
:109100000101536F0AD025C951F1020E0101536FBD
:10911000526F03D009013CD0010103D0090138D0BE
:109120000101535310E14F510901215DD8A402D030
:10913000010109D04FC121F921C928F90001B4EC7E
:109140002AF024D00101532D10D050510901215D86
:10915000D8A402D0010109D050C121F921C928F9B0
:109160000001B4EC2AF012D00101535102080FE1C2
:1091700051510901215DD8A402D0010108D051C18B
:1091800021F921C928F90001B4EC2AF001010901F3
:1091900000011CEF49F044A819D00901202B2051EF
:1091A0007C08D8A002D0000111D0236B235100010C
:1091B000FAEC0CF0000908E00901232B246F0001F0
:1091C000D8D50901F3D700010901206B040114511E
:1091D000000103E0010A08E000D00301946B0401E0
:1091E0001B6B010E146F000104011A51195D2FE071
:1091F0001A511A2B940FE96E020EEA6ED8B0EA2AC1
:10920000EFCF22F9090104011B511B2B036A940FB4
:10921000E96E030E0320EA6E22C9EFFF036A1B51B9
:10922000940FE96E030E0320EA6EEF6A09012251E2
:109230003B0806E100017DD60401146B1B6B08D0CE
:1092400004011B513E0802E2146B02D0CED700D0BD
:10925000000142EF64F00901236B45520DE04650D6
:109260001F0B236F4550020802E1238D04D04550A7
:10927000030801E1238F456A23C901F0000154EF7F
:1092800056F044A20BD0850EB16E85C0B3FF84C0EA
:10929000B2FFA082010EA76F770EA66FB1EF49F063
:1092A0004850F00B0901246F00016F9373532DE0B8
:1092B00091846F51701128E1BC5305E1BD5303E166
:1092C0002AEC34F021D0BC3D03D0BD3D01D00AD002
:1092D000BC51D8B4BD07BC2F05D0BD5303E1FDEC94
:1092E00034F012D06D5310E06D5103080DE0080109
:1092F000F72BD8B4F82BF85303E1F751180803E221
:109300008E7EF86BF76B000108D09194FDEC34F081
:109310006F51701102E18E8E8A9409012451500818
:1093200042E000016F5170113EE049523CE10901F9
:10933000239141B223812C6AF2BC2C8CF29CF2BEA8
:109340002C8EF29E000132EC0EF02CBCF28C2CBE66
:10935000F28E8E9E8A840901245130080AE00001B1
:1093600090D786C025F90901266B0001A9EC27F0EA
:1093700009012451200802E1300E486E276B0001DC
:10938000CBEC19F001520FE06E530DE10901276B90
:109390000001CBEC19F001C06EF00801F46B4296AD
:1093A000090123B14286000181EF56F009012751DE
:1093B0001208D8A0C3D027510C0DF3502B6B2A6F85
:1093C0002BC903F02A51F2CF2CF9F29CF29E000136
:1093D00008EC0BF009012CBDF28C2CBFF28E296F2A
:1093E000020E295DE30FD8B0A9D01D0F0001A2EF36
:1093F0004AF028C92AF909012B6B00014DEC19F03C
:1094000001509ED028C92AF913EC40F0015098D0A1
:1094100028C92DF922EC16F0015092D028C92DF957
:10942000F3EC16F001508CD028C92DF967EC17F039
:10943000015086D028C92AF909012B6B000133ECB1
:109440001AF001507DD028C92AF96EEC1BF00150AA
:1094500077D028C92AF909012B6B000134EC1CF0E4
:1094600001506ED028C92AF909012B6B000148EC84
:109470001DF0015065D028C92DF909012E6B00019E
:1094800014EC1EF001505CD028C92AF909012B6B9D
:109490000001CBEC1EF0015053D028C92AF9090174
:1094A0002B6B00012BEC1FF001504AD028C92AF980
:1094B00009012B6B0001A4EC1FF0015041D028C919
:1094C0002BF909012D6B2C6B0001FBEC1FF00150F7
:1094D00037D028C92AF909012C6B2B6B00010EEC3F
:1094E00022F001502DD028C92AF909012B6B000167
:1094F000EAEC23F0015024D028C92AF91BEC26F00D
:1095000001501ED028C92AF909012B6B0001EAEC91
:109510003DF0015015D028C92AF909012B6B000133
:1095200050EC24F001500CD028C92AF909012B6B0A
:109530000001DBEC24F0015003D00901000E016EA4
:109540000001000CF2CF21F0F29CF29EE824F76AB1
:10955000F736750FF66E950EF722000EF86EFB6E5D
:109560000A00F550FA6E0800F55021BCF28C21BEBD
:10957000F28EF96E04943A953A9510941C942894BE
:1095800034944694529464943A95769488949A9438
:10959000F2933A953A953A953A95AC943A95BE94A9
:1095A000D2943A95E694F894169528950495090175
:1095B00025510C0DF350286B276F28C903F0275154
:1095C000F2CF29F9F29CF29E000108EC0BF00901A0
:1095D00029BDF28C29BFF28E016E080A000103E05A
:1095E0001F0A01E01DD025C927F9030E0901286FC4
:1095F0000001DCDE26C928F9B4EC2AF00901326B3F
:109600008A0E316F336B070E346F0001C7EC17F011
:1096100025C927F9060E0901286F0001C7DE05D00C
:1096200026C928F9B4EC2AF000D0000C0901245115
:10963000000147E0080A46E0400A44E0410AD8B485
:10964000BCD0400AD8B4B9D0430AD8B418D1400A23
:10965000D8B415D1C00AD8B412D18E0AD8B484D1E6
:10966000400AD8B481D1C00AD8B47ED1820AD8B415
:10967000EFD1030AD8B4FFD11D0AD8B4FCD1080A2F
:10968000D8B4FAD1010AD8B405D2080AD8B410D295
:109690000B0AD8B419D2080AD8B424D2160AD8B4FE
:1096A0002FD2180AD8B43AD2190AD8B445D2180A17
:1096B000D8B450D21B0AD8B45BD2180AD8B466D238
:1096C00073D27ED26B5105E0010A30E0030A32E02A
:1096D00073D0010E6B6F0901326B8A0E316F336BE1
:1096E000070E346F0001C7EC17F00801F3510C0DA1
:1096F000F3500901266B256F020E2525016E000E21
:109700002621036E01C027F901C028F92851000164
:1097100008EC0BF0000909E00901282B326F000169
:10972000EAEC16F00901F2D7000146D06B6B010E8E
:10973000016E48D2F3C827F9030E0901286F000112
:1097400035DEF3C827F9070E0901286F00012EDE68
:10975000F3C827F90B0E0901286F000127DE010E5F
:109760006B6F0901326B8A0E316F336B070E346FEA
:109770000001C7EC17F00801F3510C0DF35009017B
:10978000266B256F020E2525016E000E2621036E25
:1097900001C027F901C028F92851000108EC0BF09D
:1097A000000909E00901282B326F0001EAEC16F0EC
:1097B0000901F2D7000100D003D26B2D1BD0020E9D
:1097C0006B6FF3C827F90A0E0901286F0001EEDD5F
:1097D0000901326B8A0E316F336B070E346F000153
:1097E000C7EC17F0F3C827F9060E0901286F00012E
:1097F000DDDD44D06B51020841E1F3C827F9030EC7
:109800000901286F0001D2DDF3C827F9070E09010D
:10981000286F0001CBDDF3C827F90B0E0901286F73
:109820000001C4DD010E6B6F0901326B8A0E316FCE
:10983000336B070E346F0001C7EC17F00801F351CA
:109840000C0DF3500901266B256F020E2525016EC4
:10985000000E2621036E01C027F901C028F9285106
:10986000000108EC0BF0000909E00901282B326F18
:109870000001EAEC16F00901F2D70001A1D16B2D2D
:1098800032D00801F307F351120802E2120EF36F0F
:109890000901326B8A0E316F336B070E346F000192
:1098A000C7EC17F00801F3510C0DF3500901266BBA
:1098B000256F020E2525016E000E2621036E01C0C4
:1098C00027F901C028F92851000108EC0BF0000924
:1098D00009E00901282B326F0001EAEC16F00901BA
:1098E000F2D700013ED06B5102083BE1F3C827F9E3
:1098F000040E0901286F000159DD0901326B8A0E3F
:10990000316F336B070E346F0001C7EC17F0F3C8EB
:1099100027F9060E0901286F000148DD0801F351FF
:109920000C0DF3500901266B256F010E2525016EE4
:10993000000E2621036E0150F2CF27F9F29CF29E11
:10994000000108EC0BF0090127BDF28C27BFF28E55
:10995000016EE8A007D0F3C827F9070E286F0001B1
:1099600025DD090100012CD16B2D31D00801F32B2D
:10997000F351120801E2F36B0901326B8A0E316F69
:10998000336B070E346F0001C7EC17F00801F35179
:109990000C0DF3500901266B256F020E2525016E73
:1099A000000E2621036E01C027F901C028F92851B5
:1099B000000108EC0BF0000909E00901282B326FC7
:1099C0000001EAEC16F00901F2D700013ED06B511C
:1099D00002083BE1F3C827F9050E0901286F0001D1
:1099E000E5DC0901326B8A0E316F336B070E346F81
:1099F0000001C7EC17F0F3C827F9060E0901286F1C
:109A00000001D4DC0801F3510C0DF3500901266B61
:109A1000256F010E2525016E000E2621036E0150D3
:109A2000F2CF27F9F29CF29E000108EC0BF009013D
:109A300027BDF28C27BFF28E016EE8A007D0F3C8D5
:109A400027F9070E286F0001B1DC09010001B8D029
:109A500041A20ED02C6AF2BC2C8CF29CF2BE2C8E51
:109A6000F29E39EC0EF02CBCF28C2CBEF28E02D0A1
:109A7000E7EC3EF0A5D0A4D0F3C825F9010E09010A
:109A8000266F000194DD010E0901286F0001B8EC7A
:109A900035F096D0F3C825F9020E0901266F0001B2
:109AA00086DD020E0901286F0001B8EC35F088D080
:109AB000F3C825F90901266B000179DD0901286B3E
:109AC0000001B8EC35F07CD0F3C825F9030E09018C
:109AD000266F00016CDD030E0901286F0001B8EC50
:109AE00035F06ED0F3C825F9040E0901266F000188
:109AF0005EDD040E0901286F0001B8EC35F060D07E
:109B0000F3C825F9050E0901266F000150DD050E89
:109B10000901286F0001B8EC35F052D0F3C825F9DF
:109B2000060E0901266F000142DD060E0901286FAD
:109B30000001B8EC35F044D0F3C825F9070E09014F
:109B4000266F000134DD070E0901286F0001B8EC13
:109B500035F036D0F3C825F9080E0901266F00014B
:109B600026DD080E0901286F0001B8EC35F028D079
:109B7000F3C825F9090E0901266F000118DD090E49
:109B80000901286F0001B8EC35F01AD0F3C825F9A7
:109B90000A0E0901266F00010ADD0A0E0901286F6D
:109BA0000001B8EC35F00CD06B6BF3C827F9030E4D
:109BB0000901286F0001D6EC49F0010E016E02D0B8
:109BC000000E016E000C735308E08851080803E092
:109BD0002AEC34F002D0FDEC34F097EF4EF0485010
:109BE000200A06E0010A25E0030AD8B46DD179D134
:109BF0000901326B8A0E316F336B070E346F00012F
:109C0000C7EC17F0210E486E44BC0ED02C6AF2BC93
:109C10002C8CF29CF2BE2C8EF29E32EC0EF02CBC00
:109C2000F28C2CBEF28E04D0875302E0D3EC3EF0CF
:109C300058D1040E0901235DAB0FD8B043D1550FA5
:109C4000000173EF4FF0400E486E41A20DD02C6A18
:109C5000F2BC2C8CF29CF2BE2C8EF29E32EC0EF0FA
:109C60002CBCF28C2CBEF28E919C8B9209013F6B26
:109C7000070E3E6F86C040F9000111EC12F0090199
:109C800021D1886B09011ED18851040803E0040E1C
:109C9000886F01D0886B090115D18851050803E050
:109CA000050E886F01D0886B09010CD1885102081C
:109CB00003E0020E886F01D0886B090103D1447064
:109CC0000C0E896FA56B7D0EA46F0901FBD0882D4A
:109CD00001D003D0010E886F01D0886B0901F2D04A
:109CE000220E486E23C924F9A1DC060E886F0901F3
:109CF000E9D08851030803E0030E886F01D0886B18
:109D00000901E0D041A20ED02C6AF2BC2C8CF29C4E
:109D1000F2BE2C8EF29E39EC0EF02CBCF28C2CBED6
:109D2000F28E02D0E7EC3EF00901CCD04CD709010D
:109D3000C9D0010E0901286F0001B8EC35F00152BD
:109D400006E1010E0901286F0001B4EC2AF0886BCE
:109D50000901B8D0020E0901286F0001B8EC35F0F6
:109D6000015206E1020E0901286F0001B4EC2AF04D
:109D7000886B0901A7D00901286B0001B8EC35F008
:109D8000015205E10901286B0001B4EC2AF0886B4F
:109D9000090198D0030E0901286F0001B8EC35F0D5
:109DA000015206E1030E0901286F0001B4EC2AF00C
:109DB000886B090187D0040E0901286F0001B8ECF7
:109DC00035F0015206E1040E0901286F0001B4ECE0
:109DD0002AF0886B090176D0050E0901286F000171
:109DE000B8EC35F0015206E1050E0901286F0001BB
:109DF000B4EC2AF0886B090165D0060E0901286FC2
:109E00000001B8EC35F0015206E1060E0901286F99
:109E10000001B4EC2AF0886B090154D0070E090147
:109E2000286F0001B8EC35F0015206E1070E090178
:109E3000286F0001B4EC2AF0886B090143D0080EAA
:109E40000901286F0001B8EC35F0015206E1080E57
:109E50000901286F0001B4EC2AF0886B090132D0A7
:109E6000090E0901286F0001B8EC35F0015206E136
:109E7000090E0901286F0001B4EC2AF0886B090172
:109E800021D00A0E0901286F0001B8EC35F001520B
:109E900006E10A0E0901286F0001B4EC2AF0886B74
:109EA000090110D00B0E0901286F0001B8EC35F044
:109EB000090108D00B0E0901286F0001B8EC35F03C
:109EC000090100D000010DD023C924F916EC4BF094
:109ED000015204E0210E486E886B02D0060E886F96
:109EE00000D0B2EF56F0F2CF21F0F29CF29EE824BF
:109EF000F76AF736170FF66E9F0EF722000EF86E10
:109F0000FB6E0A00F550FA6E0800F55021BCF28C89
:109F100021BEF28EF96E889C2C9D049DC49ECE9C21
:109F2000F29CAC9CC49ED89D1C9E609EC49E329D9B
:109F3000549D949DC49EFA9D3E9E829EC49EA49E66
:109F4000769DB69DC49E469CC49EC49EC49EC49EDF
:109F5000C49EC49EC49EC49EC49EC49EC49EC49EF1
:109F6000C49EC49EC49EC49EC49EC49EC49EC49EE1
:109F7000C49EC49EC49EC49EC49EC49EC49EC49ED1
:109F8000C49EC49EC49EC49EC49EC49EC49EC49EC1
:109F9000C49EC49EC49E9A9CC49EC49EC49EE09CC3
:109FA000829CBE9CC49EC49EC49EC49EC49EC49EED
:109FB000C49EC49EC49EC49EC49EC49EC49EB49EA1
:109FC00084A8B9D084500F0B0901236F07015251A7
:109FD0000901235DD8A4ABD00701532B53510308CB
:109FE000D8B0A3D0040E536F090123510F0855E1D7
:109FF00041AA01D0419C419A0F0E0701516F526F47
:10A0000048A710D02C6AF2BC2C8CF29CF2BE2C8E8D
:10A01000F29E000132EC0EF02CBCF28C2CBEF28EC3
:10A020003AD007010001872D12D0070155510308CE
:10A03000D8B002D000010BD006E15451E708D8B0E7
:10A0400002D0000104D0010E556FF40E546F0701C9
:10A0500055C703F05451542BD8B4552B0901246F24
:10A0600003C025F92451F40815E1252D13D0000E65
:10A0700041B2010E246F000E44BC010E241104E015
:10A080000001D3EC3EF04380030E0701556FE80E4C
:10A09000546F0901000138D009010701488741BA0E
:10A0A00034D0418A51510F0830E141BC2ED02C6A86
:10A0B000F2BC2C8CF29CF2BE2C8EF29EFE0E09019C
:10A0C000616F00010CEC0EF02CBCF28C2CBEF28EF9
:10A0D0002C6AF2BC2C8CF29CF2BE2C8EF29E310EBD
:10A0E0000901616F00010CEC0EF02CBCF28C2CBE4F
:10A0F000F28E418C439041B202D044AC03D0E7ECE5
:10A100003EF043800F0E866F070151510901235D18
:10A110000BE023510A0808E323C951F751C728F976
:10A120000001B4EC2AF00901070105D0090123C997
:10A1300052F70701536B0001BDEF56F084A822D1FE
:10A14000BB51010828E2FF0A03E1BA51000823E2EB
:10A15000B8350901266F0001B9350901276F263787
:10A160002737263727372637273726372737263703
:10A170002737C00E261727C951F926C950F9BBC089
:10A1800053F9BAC052F9000121EC15F002C024F9CC
:10A1900001C023F929D0BB5326E1BA51090823E3B2
:10A1A000B8350901266F0001B9350901276F263737
:10A1B00027372637273726372737263727372637B3
:10A1C0002737C00E261727C951F926C950F9030EA3
:10A1D000536F200E526F000121EC15F002C024F9DC
:10A1E00001C023F901D0CED056C725F90901245367
:10A1F00006E12351080803E3040E256FB7D024536A
:10A2000019E123510E0816E30701565104080EE127
:10A21000090123510908D8B402D0070107D02453FB
:10A22000D8B402D0070102D0040E02D00A0E0901F0
:10A23000256F9CD0245319E12351120816E307011E
:10A2400056510A080EE1090123510F08D8B402D073
:10A25000070107D02453D8B402D0070102D00A0E58
:10A2600002D0090E0901256F81D0245319E1235131
:10A270001A0816E30701565109080EE10901235196
:10A280001308D8B402D0070107D02453D8B402D0A1
:10A29000070102D0090E02D0070E0901256F66D012
:10A2A000245319E12351220816E3070156510708E8
:10A2B0000EE1090123511B08D8B402D0070107D0D1
:10A2C0002453D8B402D0070102D0070E02D0050EE5
:10A2D0000901256F4BD0245319E123512A0816E3B5
:10A2E0000701565105080EE1090123512308D8B48E
:10A2F00002D0070107D02453D8B402D0070102D0FE
:10A30000050E02D0030E0901256F30D0245319E148
:10A310002351320816E30701565103080EE10901E3
:10A3200023512B08D8B402D0070107D02453D8B446
:10A3300002D0070102D0030E02D0020E0901256FE0
:10A3400015D00701565102080EE1090123513308C7
:10A35000D8B402D0070107D02453D8B402D00701E3
:10A3600002D0020E02D0010E0901256F07015651DD
:10A370000901255D08E025C956F756C728F90001EF
:10A38000B4EC2AF009010001BDEF56F09D9A9D98AA
:10A39000B8EF52F0A39AA398B9EF52F08A90020E48
:10A3A00009012B6FC69A2B2D03D0300EC66E02D03A
:10A3B000320EC66EC76AC68A0D0E006E002EFED71C
:10A3C0009198919E020E006E002EFED70000316B18
:10A3D000C9CF32F931C9C9FFC7A0FED7C9CF32F9F9
:10A3E000326B3251010802E3322BFBD7316BC9CFFC
:10A3F00032F931C9C9FFC7A0FED7C9CF32F9326BD4
:10A400003251010802E3322BFBD7316BC9CF32F94D
:10A4100031C9C9FFC7A0FED7C9CF32F9326B32515B
:10A42000010802E3322BFBD7316BC9CF32F931C9B6
:10A43000C9FFC7A0FED7C9CF32F9326B325101082C
:10A4400002E3322BFBD7020E006E002EFED7000077
:10A45000918E9188010E2B6FC69A2B2D03D0300E52
:10A46000C66E02D0320EC66EC76AC68A0D0E006E68
:10A47000002EFED70001D5EF52F0030E09012D6F1B
:10A48000000122EC16F0030E09012D6F0001F3EC20
:10A4900016F0030E09012D6F000167EC17F0030E93
:10A4A0000901276F0001CBEC19F0030E09012A6F97
:10A4B000FF0E2B6F000133EC1AF0030E09012A6F17
:10A4C00000016EEC1BF0030E09012A6F2B6B0001DB
:10A4D00034EC1CF0030E09012A6F2B6B000148ECD1
:10A4E0001DF0030E09012D6F2E6B000114EC1EF000
:10A4F000030E09012A6F2B6B0001CBEC1EF0030E3B
:10A5000009012A6F2B6B00012BEC1FF0030E0901D0
:10A510002A6F2B6B0001A4EC1FF0030E09012A6FB8
:10A520002B6B0001EAEC23F0030E09012A6F2B6B61
:10A53000000150EC24F0030E09012A6F2B6B00017F
:10A54000DBEC24F0EEEF52F02C6AF2BC2C8CF29C87
:10A55000F2BE2C8EF29E32EC0EF02CBCF28C2CBE95
:10A56000F28E919609012E6B000145EC24F00ED776
:10A5700011D72C6AF2BC2C8CF29CF2BE2C8EF29E6F
:10A58000320E0901616F00010CEC0EF02CBCF28C54
:10A590002CBEF28E9EEC22F0AEEC3BF0FE0E0901DA
:10A5A000286F0001D0EC3BF0F9D6C80E0901286FE6
:10A5B00000011FEC10F009013F6B090E3E6F44C013
:10A5C00040F9000111EC12F009013F6BFD0E3E6FE6
:10A5D000FF0E406F000111EC12F04FD79080908277
:10A5E0009094909684AC04D0875309E1535207E0CD
:10A5F000010E0901286F00011FEC10F0F3D7FF00D6
:10A60000C2EF56F00901326B8A0E316F336B070EC1
:10A61000346F0001C7EC17F009012551020A00014F
:10A6200021E0010A31E0070A41E0020A51E0010A93
:10A6300061E00F0AD8B470D0010AD8B47FD0030A01
:10A64000D8B48ED0010AD8B49DD0070AD8B4ACD003
:10A65000030AD8B4BBD0020AD8B4CAD0030AD8B40B
:10A66000D9D0EAD00901266B265100018CEC0BF001
:10A67000000909E00901262B326F0001EAEC16F00F
:10A680000901F2D70001EAD00901266B2651000129
:10A69000A3EC0BF0000909E00901262B326F000141
:10A6A000EAEC16F00901F2D70001D8D00901266BB7
:10A6B00026510001BAEC0BF0000909E00901262B34
:10A6C000326F0001EAEC16F00901F2D70001C6D0A2
:10A6D0000901266B26510001D1EC0BF0000909E0BD
:10A6E0000901262B326F0001EAEC16F00901F2D7BE
:10A6F0000001B4D00901266B26510001E8EC0BF0F3
:10A70000000909E00901262B326F0001EAEC16F07E
:10A710000901F2D70001A2D00901266B26510001E0
:10A72000FFEC0BF0000909E00901262B326F000154
:10A73000EAEC16F00901F2D7000190D00901266B6E
:10A740002651000116EC0CF0000909E00901262B46
:10A75000326F0001EAEC16F00901F2D700017ED059
:10A760000901266B265100012DEC0CF0000909E0CF
:10A770000901262B326F0001EAEC16F00901F2D72D
:10A7800000016CD00901266B2651000144EC0CF04D
:10A79000000909E00901262B326F0001EAEC16F0EE
:10A7A0000901F2D700015AD00901266B2651000198
:10A7B0005BEC0CF0000909E00901262B326F000167
:10A7C000EAEC16F00901F2D7000148D00901266B26
:10A7D0002651000172EC0CF0000909E00901262B5A
:10A7E000326F0001EAEC16F00901F2D7000136D011
:10A7F0000901266B2651000189EC0CF0000909E0E3
:10A800000901262B326F0001EAEC16F00901F2D79C
:10A81000000124D00901266B26510001A0EC0CF0A8
:10A82000000909E00901262B326F0001EAEC16F05D
:10A830000901F2D7000112D00901266B265100014F
:10A84000B7EC0CF0000909E00901262B326F00017A
:10A85000EAEC16F00901F2D7000100D08851080196
:10A86000F55D02E088C0F5F8070E0001886F000C66
:10A87000020E0901255DF20FD8B099D00E0F00012C
:10A88000DAEF54F0020E0901376F75C039F974C060
:10A8900038F9000145EC12F0090189D0030E0901D5
:10A8A000376F396B386B000145EC12F009017FD02E
:10A8B000040E0901376F77C039F976C038F9000105
:10A8C00045EC12F0090173D0060E0901376F79C00B
:10A8D00039F978C038F9000145EC12F0090167D068
:10A8E000070E0901376F396B386B000145EC12F028
:10A8F00009015DD0080E0901376F7BC039F97AC0B4
:10A9000038F9000145EC12F0090151D0090E090196
:10A91000376F7FC039F97EC038F9000145EC12F07D
:10A92000090145D00A0E0901376F396B386B0001F8
:10A9300045EC12F009013BD00B0E0901376F81C0C5
:10A9400039F980C038F9000145EC12F009012FD027
:10A950000C0E0901376F7DC039F97CC038F9000150
:10A9600045EC12F0090123D00F0E0901376F83C0A7
:10A9700039F982C038F9000145EC12F0090117D00D
:10A980000D0E0901376F7BC039F97AC038F9000123
:10A9900045EC12F009010BD00E0E0901376F396B2F
:10A9A000386B000145EC12F0090101D009010001EA
:10A9B000C2EF55F0F2CF21F0F29CF29EE824F76A44
:10A9C000F736E50FF66EA90EF722000EF86EFB6E55
:10A9D0000A00F550FA6E0800F55021BCF28C21BE39
:10A9E000F28EF96E84A89CA8B0A8ACA9C8A8E0A86B
:10A9F000F4A80CA924A938A950A980A998A968A9E4
:10AA00000901246B4850320A000103E0020A0CE0FD
:10AA10001ED1300E486E6CC025F9F4DD09012351BA
:10AA20004808D8B4236B00016C53D8A4BED072BBC5
:10AA300008D070AB06D00D0E0901246F0001728B97
:10AA400077D072B908D070A906D00E0E0901246F14
:10AA5000000172896DD072B708D070A706D00F0EB2
:10AA60000901246F0001728763D071B508D06FA50A
:10AA700006D0040E0901246F0001718559D071B10F
:10AA800008D06FA106D0020E0901246F0001718168
:10AA90004FD071B308D06FA306D0030E0901246F05
:10AAA0000001718345D071B908D06FA906D0060E98
:10AAB0000901246F000171893BD072B308D070A3E3
:10AAC00006D00B0E0901246F0001728331D071BDD5
:10AAD00008D06FAD06D0080E0901246F0001718DFA
:10AAE00027D072B508D070A506D00C0E0901246FCE
:10AAF000000172851DD071BF08D06FAF06D0090E5E
:10AB00000901246F0001718F13D072B108D070A1B8
:10AB100006D00A0E0901246F0001728109D071BBB1
:10AB200007D06FAB05D0070E0901246F0001718BB0
:10AB300072C003F0031E7151FF0A6F15006E0350BF
:10AB40007015036E0050031002E1726B716B090106
:10AB500024532CE024C96CF02C6AF2BC2C8CF29C9F
:10AB6000F2BE2C8EF29E000132EC0EF02CBCF28C68
:10AB70002CBEF28E8E9E8A8424C925F943DD24C919
:10AB800025F976D6090124512009256F2C6AF2BCDB
:10AB90002C8CF29CF2BE2C8EF29E616F00010CECAC
:10ABA0000EF02CBCF28C2CBEF28E09010001A651D5
:10ABB000A71109E0A651D8B4A707A62F04D0A75320
:10ABC00002E19EEC22F06E5313E00801F42BF451E5
:10ABD0007C080FE2F46B00016E2F0AD01EEC3BF0F4
:10ABE0006F51701104E142A602D0E7EC3EF02FD085
:10ABF000080109012351060A000107E0030A0DE0DC
:10AC00004D0A0EE0540A11E022D01EEC3BF06F51C9
:10AC1000701102E1E7EC3EF01AD01EEC3BF017D0C9
:10AC2000320E486E010E6B6F12D01EEC3BF0400EE0
:10AC3000486E2C6AF2BC2C8CF29CF2BE2C8EF29EDA
:10AC400032EC0EF02CBCF28C2CBEF28E00D0D4EF85
:10AC500056F00701436B0901246B24510001E5EC18
:10AC60000CF0000911E00901242B3B6F070143514F
:10AC7000432B036AAC0FE96E060E0320EA6E3BC954
:10AC8000EFFF0901EAD7000109012B6B23C92AF95B
:10AC9000030E2C6F2D6B0001E8EC32F023EC33F047
:10ACA000D3EF56F02BEF49F001C022F9895110087B
:10ACB0000DE1A451A5110AE009012253D8A402D044
:10ACC000000104D00001A56BA46B896B475208E01A
:10ACD000472E06D088A002D0708902D0D3EC3EF077
:10ACE00087530DE142AA0BD0535206E053500A0895
:10ACF00003E053500C0803E1D3EC3EF0429A50EFCE
:10AD000049F00901286B0001D0EC3BF04850F00BF2
:10AD1000100A09E0300A22E0600A30E0700A33E0ED
:10AD2000600A34E041D041A618D02C6AF2BC2C8CC9
:10AD3000F29CF2BE2C8EF29E32EC0EF02CBCF28C09
:10AD40002CBEF28E8651F0090901236F256F266B08
:10AD50000001A9EC27F0200E486E26D022C923F965
:10AD6000EFEF4DF08751FC0F08E2040FD6EF56F0DD
:10AD7000E0EF4FF09EEF50F000D016D042B202D07C
:10AD8000A4EF52F011D022C923F93AD64850510805
:10AD90000AE109012253D8A402D0000104D022C93B
:10ADA00023F9000156D700D044EF64F0F2CF21F030
:10ADB000F29CF29EE824F76AF736DD0FF66EAD0ED0
:10ADC000F722000EF86EFB6E0A00F550FA6E0800CE
:10ADD000F55021BCF28C21BEF28EF96E70AD70ADD3
:10ADE00074AD78ADF00E67176817C00E69176A1753
:10ADF000000C0F0E671768173F0E6917000C4BC940
:10AE00004BF009014C6B036A4C514925E96E4A51DC
:10AE10000320EA6EEF5218E04C51090815E3036A6B
:10AE20004C514925E96E4A510320EA6EEFCF4DF9A6
:10AE300048C94FF947C94EF94DC950F9000199EC7D
:10AE400015F009014C2BDFD70001000C639EA49E76
:10AE50003CC966FF020E63BE05D0A4AEFED7000E4D
:10AE600062BC010E016E000C010E0901396F070E64
:10AE70003B6F590E3A6F628062B0FED7700E386F2A
:10AE800038C93CF90001E2DF015217E10901396BD1
:10AE9000376B3751120810E33751372B036A3A25C5
:10AEA000E96E3B510320EA6EEFCF38F938C93CF91F
:10AEB0000001CCDF0901EDD70001628462B4FED746
:10AEC000090139C901F00001000C080E0901366FB3
:10AED000070E356F6B0E346F31C9E9FF32C9EAFFD7
:10AEE000EF503F0B336F35C903F03451D8B43507F9
:10AEF0003407E96E03C0EAFFD89033353A6B396FF7
:10AF0000010E3925016E000E3A21036E0150F2CF79
:10AF10003BF9F29CF29E0001E5EC06F009013BBD15
:10AF2000F28C3BBFF28EEF6E34C9E9FF35C9EAFF00
:10AF3000D89033353A6B396F3AC903F03951F2CFB3
:10AF40003BF9F29CF29E0001E5EC06F009013BBDE5
:10AF5000F28C3BBFF28EEF6E32C903F031C9E9FFCC
:10AF600032C9EAFFEFAC07D034C9E9FF35C9EAFFBF
:10AF7000EF508009EF6E32C903F031C9E9FF32C9E1
:10AF8000EAFFEFAE07D034C9E9FF35C9EAFFEF5059
:10AF90000109EF6E3451D8B435073407312BD8B4DA
:10AFA000322B362F99D7C80E0701596FF00E5A6F02
:10AFB0005B6B000159DF000CFF0E07016B6F6A6FBE
:10AFC000696F686F676F666F656F646F636F626FDD
:10AFD000616F606F5F6F5E6F5D6F5C6FC80E596F02
:10AFE000F00E5A6F5B6B00013FDFD7EF5BF0010E95
:10AFF0000901355DEC0F41E2140F00013FEF58F0FD
:10B00000678109013AD06783090137D06785090153
:10B0100034D06787090131D0688109012ED0688357
:10B0200009012BD06885090128D06887090125D03E
:10B030006981090122D0698309011FD0698509014D
:10B040001CD06987090119D06989090116D0698B5B
:10B05000090113D06A81090110D06A8309010DD05A
:10B060006A8509010AD06A87090107D06A8909013E
:10B0700004D06A8B090101D009010001000CF2CF54
:10B0800021F0F29CF29EE824F76AF736AF0FF66ED5
:10B09000B00EF722000EF86EFB6E0A00F550FA6E45
:10B0A0000800F55021BCF28C21BEF28EF96E72B010
:10B0B0006CB066B060B05AB054B04EB048B042B058
:10B0C0003CB036B030B02AB024B01EB018B012B0C8
:10B0D0000CB006B000B0010E0901325DEC0F19E2B0
:10B0E000140F00018CEF58F06781678367856787CD
:10B0F00068816883688568876981698369856987EC
:10B100006989698B6A816A836A856A876A896A8BB9
:10B110000901000168EF5CF0F2CF21F0F29CF29E91
:10B12000E824F76AF736490FF66EB10EF722000EE3
:10B13000F86EFB6E0A00F550FA6E0800F55021BC5F
:10B14000F28C21BEF28EF96E0EB10CB10AB108B1CB
:10B1500006B104B102B100B1FEB0FCB0FAB0F8B073
:10B16000F6B0F4B0F2B0F0B0EEB0ECB0EAB0E8B0E7
:10B170000901315107016C5D03E06D6B31C96CF75A
:10B1800009013E6B3BC13DF9406B0C0E3F6F000166
:10B19000ABEC11F002C034F901C033F90B0E090118
:10B1A0000124016E000E0220036E0150F2CF35F92A
:10B1B000F29CF29E03C0F7FF0001C2EC04F009010B
:10B1C00035BDF28C35BFF28E326F07016D516D2B9C
:10B1D000FC0F28E2040F000119EF59F031C935F9CD
:10B1E00006DF07011FD009013251030804E231C90B
:10B1F00035F90001FCDE070115D0090132510008C4
:10B2000004E231C935F90001F2DE07010BD0090172
:10B210003251060804E231C935F90001E8DE0701C0
:10B2200001D007016D51040801E26D6B00016BEF65
:10B230005CF0F2CF21F0F29CF29EE824F76AF73638
:10B24000630FF66EB20EF722000EF86EFB6E0A0068
:10B25000F550FA6E0800F55021BCF28C21BEF28E3A
:10B26000F96EDCB1E6B1FAB10EB201014A5303E165
:10B270004951090803E20001698D01014A5303E1C4
:10B2800049510B0803E20001698F01014A5303E1B0
:10B2900049510C0803E20001688901014A5303E1A6
:10B2A00049510E0803E20001688B01014A5303E192
:10B2B0004951100803E20001688D01014A5303E17E
:10B2C0004951130803E20001688F01014A5303E169
:10B2D0004951180803E20001678901014A5303E15B
:10B2E00049511D0803E20001678B01014A5303E144
:10B2F0004951270803E20001678D01014A5303E128
:10B300004951310803E20001678F010100016CEF30
:10B310005CF0090E09013E6F000186510F0B010A16
:10B320001CE0030A31E0020A46E0030A5BE0070A78
:10B33000D8B46FD0010AD8B483D0030AD8B497D058
:10B34000010AD8B4ABD00F0AD8B4BFD0010AD8B420
:10B35000D3D0030AD8B4E7D0FED0090EEA6E340E7B
:10B36000E96EF2CF3FF9F29CF29E000E37EC07F047
:10B370000A000900F550EE6E0009FBE109013FBD2E
:10B38000F28C3FBFF28E00D1090EEA6E340EE96EE8
:10B39000F2CF3FF9F29CF29E000E4EEC07F00A004D
:10B3A0000900F550EE6E0009FBE109013FBDF28C8A
:10B3B0003FBFF28EE9D0090EEA6E340EE96EF2CF8D
:10B3C0003FF9F29CF29E000E65EC07F00A000900BE
:10B3D000F550EE6E0009FBE109013FBDF28C3FBF65
:10B3E000F28ED2D0090EEA6E340EE96EF2CF3FF93A
:10B3F000F29CF29E000E7CEC07F00A000900F5506A
:10B40000EE6E0009FBE109013FBDF28C3FBFF28EF9
:10B41000BBD0090EEA6E340EE96EF2CF3FF9F29C12
:10B42000F29E000E93EC07F00A000900F550EE6E54
:10B430000009FBE109013FBDF28C3FBFF28EA4D0B1
:10B44000090EEA6E340EE96EF2CF3FF9F29CF29EDD
:10B45000000EAAEC07F00A000900F550EE6E000994
:10B46000FBE109013FBDF28C3FBFF28E8DD0090E8A
:10B47000EA6E340EE96EF2CF3FF9F29CF29E000EB6
:10B48000C1EC07F00A000900F550EE6E0009FBE17F
:10B4900009013FBDF28C3FBFF28E76D0090EEA6EF5
:10B4A000340EE96EF2CF3FF9F29CF29E000ED8EC1A
:10B4B00007F00A000900F550EE6E0009FBE10901F2
:10B4C0003FBDF28C3FBFF28E5FD0090EEA6E340EA4
:10B4D000E96EF2CF3FF9F29CF29E000EEFEC07F01E
:10B4E0000A000900F550EE6E0009FBE109013FBDBD
:10B4F000F28C3FBFF28E48D0090EEA6E340EE96E30
:10B50000F2CF3FF9F29CF29E000E06EC08F00A0022
:10B510000900F550EE6E0009FBE109013FBDF28C18
:10B520003FBFF28E31D0090EEA6E340EE96EF2CFD3
:10B530003FF9F29CF29E000E1DEC08F00A00090093
:10B54000F550EE6E0009FBE109013FBDF28C3FBFF3
:10B55000F28E1AD00001090EEA6E340EE96EF2CFB7
:10B560003FF9F29CF29E000E34EC08F00A0009004C
:10B57000F550EE6E0009FBE109013FBDF28C3FBFC3
:10B58000F28E080E3E6F00D032C941F931C940F940
:10B59000090E436F340E426F446B3EC945F90001FA
:10B5A000DBEC15F0A2EF5CF00901366B32C948F90B
:10B5B00031C947F9090E4A6F370E496F050E4B6FB7
:10B5C0004C6B4D6B000144EC15F033C94BF0090195
:10B5D0003651362B036A3D0FE96E090E0320EA6EE1
:10B5E00037C9EFFF3651362B036A3D0FE96E090E5E
:10B5F0000320EA6E38C9EFFF35530AE03651362B87
:10B60000036A3D0FE96E090E0320EA6E2E0EEF6EFF
:10B61000345102080AE23651362B036A3D0FE96EB7
:10B62000090E0320EA6E39C9EFFF345103080AE21C
:10B630003651362B036A3D0FE96E090E0320EA6E80
:10B640003AC9EFFF345104080AE23651362B036A37
:10B650003D0FE96E090E0320EA6E3BC9EFFF036A56
:10B6600036513D0FE96E090E0320EA6EEF6A486B12
:10B670008A0E476F090E4A6F3D0E496F33C94BF969
:10B680000001FFEC56F035EF5FF009014F6B8A0EB9
:10B690004E6F31C950F9000199EC15F0000C48507B
:10B6A000510A06E0030A3FE0010AD8B479D081D0FC
:10B6B000F2EC56F0F9EC56F0E4EC17F026C932F94A
:10B6C00025C931F90901336B070E346F0001C7EC4E
:10B6D00017F0090EEA6E270EE96EF2CF31F9F29CEF
:10B6E000F29E000E4BEC08F00A000900F550EE6ED9
:10B6F0000009FBE1090131BDF28C31BFF28E26C990
:10B7000048F925C947F9090E4A6F270E496F4B6B57
:10B710000001FFEC56F026C932F925C931F965EC74
:10B7200057F062EF60F026C932F925C931F90901F5
:10B73000336B070E346F0001C7EC17F0090EEA6E89
:10B74000270EE96EF2CF31F9F29CF29E000E62EC08
:10B7500008F00A000900F550EE6E0009FBE109014E
:10B7600031BDF28C31BFF28E26C948F925C947F99F
:10B77000090E4A6F270E496F4B6B0001FFEC56F024
:10B7800026C932F925C931F965EC57F0FF0E6A6F09
:10B79000696F686F676F8E9EE4EC17F062EF60F080
:10B7A000F2EC56F0F9EC56F0E4EC17F005D462EF49
:10B7B00060F00901249141A2248144AA1DD041A234
:10B7C00013D084B808D04B0E01013B6F4A6B0A0EB0
:10B7D000496F05D0090101013B6B4A6B496B0001C0
:10B7E0006A8D6A9F08D0090101013B6B4A6B496B66
:10B7F00000016A9D6A8F09013E6B3BC13DF9406BB8
:10B800000C0E3F6F0001ABEC11F002C032F901C029
:10B8100031F90A0E09010124016E000E0220036EA7
:10B820000150F2CF33F9F29CF29E03C0F7FF000102
:10B83000C2EC04F0090133BDF28C33BFF28E226FEB
:10B840000001F2EC56F0F9EC56F044A03AD00701B2
:10B85000845101013B5D05E33BC184F7960E07016E
:10B86000816F070181532CE009013E6B84C73DF9CC
:10B87000406B0C0E3F6F0001ABEC11F002C032F9CF
:10B8800001C031F90A0E09010124016E000E0220E7
:10B89000036E0150F2CF33F9F29CF29E03C0F7FF22
:10B8A0000001C2EC04F0090133BDF28C33BFF28E0B
:10B8B000346F356F0001F7EC57F00701810701D0B5
:10B8C000846B010E0901225D316F326F000103D4D8
:10B8D00022C931F94DD4C9D4E4EC17F0A451A51113
:10B8E0000FE0A451D8B4A507A407A451A51108E0FE
:10B8F00089C023F90901266B920E256F08D000013B
:10B90000896B88C023F90901266B8A0E256F2351A4
:10B91000EF0FD8B043EF60F0110F000164EF60F05B
:10B9200026C932F925C931F90901336B070E346F85
:10B930000001C7EC17F026C932F925C931F986C0D4
:10B9400033F9E7D409019FD344A026D0B3510701AE
:10B95000755D0FE308E174510001B25DD8A002D01B
:10B96000070107D00701B3C075F7B2C074F7640EC2
:10B97000836F7435726F7535736F723773377237C3
:10B980007337F80E7217835302E0830703D0FF0E5C
:10B99000756F746F08D00001B25107017227000162
:10B9A000B35107017323802B8051070860E2040E16
:10B9B00072250901316F000E070173210901326FF1
:10B9C00032310701736F090131310701726F73332F
:10B9D0007233733372331F0E731773C73EF972C716
:10B9E0003DF90901406B0A0E3F6F0001ABEC11F00D
:10B9F000090102300701736F090101300701726FFD
:10BA0000733372337333723373337233733372330A
:10BA1000070E731726C932F925C931F90901336BAD
:10BA2000346F0001C7EC17F00901316B315100018F
:10BA300079EC08F0000909E00901312B326F0001AF
:10BA4000EAEC16F00901F2D7000173C732F972C7A8
:10BA500031F9050E0901336F030E346F010E356F96
:10BA60000001EDEC21F00701736B726B806B090133
:10BA70000AD326C932F925C931F90901336B070EFA
:10BA8000346F0001C7EC17F00901316B315100012F
:10BA90008DEC08F0000909E00901312B326F00013B
:10BAA000EAEC16F00901F2D70001ABC032F9AAC0E6
:10BAB00031F9050E0901336F020E346F356B000149
:10BAC000EDEC21F00901DFD244A028D0070171512B
:10BAD0000001B15D10E308E1B0510701705DD8A02D
:10BAE00002D0000108D00001B1C071F7B0C070F7FA
:10BAF000640E0701826F070170356E6F71356F6FCD
:10BB00006E376F376E376F37F80E6E17825302E05D
:10BB1000820702D0716B706B08D00001B051070131
:10BB20006E270001B15107016F237F2B7F5107085A
:10BB300053E2040E6E250901316F000E07016F21DB
:10BB40000901326F323107016F6F0901313107018D
:10BB50006E6F6F336E336F336E331F0E6F176FC799
:10BB60003EF96EC73DF90901406B0A0E3F6F0001B7
:10BB7000ABEC11F002C06EF707016F6B26C932F90A
:10BB800025C931F90901336B070E346F0001C7EC89
:10BB900017F00901316B31510001A4EC08F00009E4
:10BBA00009E00901312B326F0001EAEC16F00901BE
:10BBB000F2D700016FC732F96EC731F9050E0901DE
:10BBC000336F030E346F010E356F0001EDEC21F081
:10BBD00007016F6B6E6B7F6B090155D244A02CD0AF
:10BBE00009013E6B84C73DF9406B0C0E3F6F0001AD
:10BBF000ABEC11F002C032F901C031F9060E0901B7
:10BC00000124016E000E0220036E0150F2CF33F9C1
:10BC1000F29CF29E03C0F7FF0001C2EC04F00900A1
:10BC2000F5CF03F0090133BDF28C33BFF28E07016B
:10BC300078270350792308D001014B510701782759
:10BC400001014C51070179237D2B7D51030841E20D
:10BC5000020E78250901316F000E070179210901D3
:10BC6000326F32310701796F090131310701786F85
:10BC7000793378333F0E791726C932F925C931F95E
:10BC80000901336B070E346F0001C7EC17F009018F
:10BC9000316B31510001B9EC08F0000909E00901EC
:10BCA000312B326F0001EAEC16F00901F2D70001E6
:10BCB00079C732F978C731F9050E0901336F030EE0
:10BCC000346F356B0001EDEC21F00701796B786B77
:10BCD0007D6B0901D8D10101495107017A27010182
:10BCE0004A5107017B237C2B7C5107084AE2040E52
:10BCF0007A250901316F000E07017B210901326F9E
:10BD0000323107017B6F0901313107017A6F7B33D3
:10BD10007A337B337A331F0E7B1726C932F925C954
:10BD200031F90901336B070E346F0001C7EC17F0CE
:10BD30000901316B31510001CEEC08F0000909E036
:10BD40000901312B326F0001EAEC16F00901F2D73C
:10BD5000000107017B5303E17A5109080FE27BC719
:10BD600032F97AC731F9050E0901336F030E346FCA
:10BD7000010E356F0001EDEC21F007017B6B7A6B52
:10BD80007C6B090180D101014D5107017625016EBF
:10BD900001014E510701772101C076F7776F7E2BA5
:10BDA0007E51070843E2040E76250901316F000E2B
:10BDB000070177210901326F32310701776F0901DD
:10BDC00031310701766F77337633773376331F0E51
:10BDD000771726C932F925C931F90901336B070EE6
:10BDE000346F0001C7EC17F00901316B31510001CC
:10BDF000E3EC08F0000909E00901312B326F000182
:10BE0000EAEC16F00901F2D7000177C732F976C7DC
:10BE100031F9050E0901336F030E346F356B0001E4
:10BE2000EDEC21F00701776B766B7E6B09012BD16E
:10BE3000010139513A1119E026C932F925C931F900
:10BE40000901336B070E346F0001C7EC17F03AC1DC
:10BE500032F939C131F9010E0901336F050E346F22
:10BE6000010E356F0001D4EF5AF009010CD126C93B
:10BE700032F925C931F90901336B070E346F00011E
:10BE8000C7EC17F044A018D0090EEA6E270EE96E31
:10BE9000F2CF31F9F29CF29E000EF8EC08F00A00A5
:10BEA0000900F550EE6E0009FBE1090131BDF28C8D
:10BEB00031BFF28E17D00001090EEA6E270EE96E2F
:10BEC000F2CF31F9F29CF29E000E0FEC09F00A005D
:10BED0000900F550EE6E0009FBE1090131BDF28C5D
:10BEE00031BFF28E26C948F925C947F9090E4A6FB4
:10BEF000270E496F4B6B0001FFEC56F00901C3D0D0
:10BF000026C932F925C931F90901336B070E346F9F
:10BF10000001C7EC17F0090EEA6E270EE96EF2CFAA
:10BF200031F9F29CF29E000E26EC09F00A0009009D
:10BF3000F550EE6E0009FBE1090131BDF28C31BF15
:10BF4000F28E26C948F925C947F9090E4A6F270E0E
:10BF5000496F4B6B0001FFEC56F0090194D026C9E4
:10BF600032F925C931F90901336B070E346F00012D
:10BF7000C7EC17F0090EEA6E270EE96EF2CF31F921
:10BF8000F29CF29E000E3DEC09F00A000900F5500B
:10BF9000EE6E0009FBE1090131BDF28C31BFF28E7A
:10BFA00026C948F925C947F9090E4A6F270E496F76
:10BFB0004B6B0001FFEC56F0090165D026C932F940
:10BFC00025C931F90901336B070E346F0001C7EC45
:10BFD00017F0090EEA6E270EE96EF2CF31F9F29CE6
:10BFE000F29E000E53EC09F00A000900F550EE6EC7
:10BFF0000009FBE1090131BDF28C31BFF28E26C987
:10C0000048F925C947F9090E4A6F270E496F4B6B4E
:10C010000001FFEC56F0090136D026C932F925C9D6
:10C0200031F90901336B070E346F0001C7EC17F0CB
:10C030009A5302E09A3D15D0EA6A9A0EE96EF2CF61
:10C0400031F9F29CF29E000E6AEC09F00A00090038
:10C05000F550EE6E0009FBE1090131BDF28C31BFF4
:10C06000F28E26C948F925C947F909014A6B9A0E8B
:10C07000496F4B6B0001FFEC56F0090104D0090138
:10C08000248101D0090124B116D04B6A44AE0BD0F3
:10C0900084BA09D084B807D05F0E316F000145EC37
:10C0A0005BF008D0090141A806D02A0E316F0001CB
:10C0B00045EC5BF0090126C932F925C931F90001C7
:10C0C00065EC57F048EF64F0F2CF21F0F29CF29E5D
:10C0D000E824F76AF736F90FF66EC00EF722000E65
:10C0E000F86EFB6E0A00F550FA6E0800F55021BCA0
:10C0F000F28C21BEF28EF96E20B948B972BAC8BA74
:10C10000DCBBD6BC7EC07EC07EC084C030BE86BDD7
:10C110006EBE00BF5EBFBCBF1AC0F86A9F80A2821D
:10C120009F9A9F98A59AA598D08E1B8EEA6AE96A75
:10C130007E96190EAF6EA60EAC6E900EAB6E7C9610
:10C14000190E6F6EA60E6C6E900E6B6E958C958AA6
:10C15000090E656E280E636E649E649CC150C00B10
:10C160000F09C16E070EB46E140EC06FC16FC26F9F
:10C17000C36FC46FC56FC66FC76FC86FC96FCA6F13
:10C18000CB6F0F0E01014F6F506F516F0701476B5F
:10C19000489148834885496B4A6B4B6B4C6B4D6BA0
:10C1A0004E6F4F6F506B516F526F536B4897546B7C
:10C1B000556B566F576B586B6C6B6D6B6E6B6F6B13
:10C1C000706B716B726B736BFF0E746F756F766B48
:10C1D000776B786B796B7A6B7B6B7C6B7D6B7E6B33
:10C1E0007F6B806B816B826B836B846B856B866BE3
:10C1F000876B886B030E896F8A6B8B6B8C6B010E60
:10C200008D6F8E6F030E8F6F906B916B926B936B34
:10C21000946B956B966B976B986B996B9A6B9B6B0A
:10C220009C6B010E9D6F9E6B9F6BA06BA16BA26BB5
:10C23000A36BA46B1E0EA56F060EA66FA76FA86B4F
:10C24000350EA96F360EAA6FAB6F370EAC6FAD6FA0
:10C25000380EAE6FAF6F390EB06FB16F3A0EB26F6E
:10C26000B36F3B0EB46FB56F3C0EB66FB76F3D0E3C
:10C27000B86F3E0EB96FBA6F3F0EBB6FBC6F400E0A
:10C28000BD6F410EBE6FBF6F420EC06F430EC16FD8
:10C29000C26F440EC36F450EC46F460EC56FC66FA6
:10C2A000470EC76F480EC86F490EC96F4A0ECA6F56
:10C2B000CB6F4B0ECC6F4C0ECD6F4D0ECE6F4E0E26
:10C2C000CF6F4F0ED06F500ED16FD26B030ED36F66
:10C2D000D46BD56BF40ED66F010ED76F600ED86F8E
:10C2E000F00ED96F260EDA6F020EDB6FCC0EDC6F0C
:10C2F000F10EDD6F580EDE6F020EDF6FFB0EE06F8A
:10C30000F20EE16F8A0EE26F020EE36FFB0EE46F36
:10C31000F30EE56FBC0EE66F020EE76FD70EE86F07
:10C32000F40EE96FEE0EEA6F020EEB6F950EEC6FF6
:10C33000F50EED6F200EEE6F030EEF6F3C0EF06FFB
:10C34000F60EF16F520EF26F030EF36FCF0EF46F15
:10C35000F60EF56F840EF66F030EF76F520EF86F40
:10C36000F70EF96FB60EFA6F030EFB6FC70EFC6F78
:10C37000F70EFD6FE80EFE6F030EFF6F300E080123
:10C38000006FF80E016F1A0E026F040E036F8F0E0E
:10C39000046FF80E056F4C0E066F040E076FE60E65
:10C3A000086FF80E096F7E0E0A6F040E0B6F350EC4
:10C3B0000C6FF90E0D6FB00E0E6F040E0F6F7D0E29
:10C3C000106FF90E116FE20E126F040E136FC00E94
:10C3D000146FF90E156F140E166F050E176FFE0E03
:10C3E000186FF90E196F460E1A6F050E1B6F370E78
:10C3F0001C6FFA0E1D6F780E1E6F050E1F6F6B0EF1
:10C40000206FFA0E216FAA0E226F050E236F9D0E6C
:10C41000246FFA0E256FDC0E266F050E276FCB0EEC
:10C42000286FFA0E296F0E0E2A6F060E2B6FF60E6E
:10C430002C6FFA0E2D6F400E2E6F060E2F6F1E0EF4
:10C44000306FFB0E316F720E326F060E336F440E7B
:10C45000346FFB0E356FA40E366F060E376F680E05
:10C46000386FFB0E396FD60E3A6F060E3B6F890E92
:10C470003C6FFB0E3D6F080E3E6F070E3F6FA90E1F
:10C48000406FFB0E416F3A0E426F070E436FC70EAF
:10C49000446FFB0E456F6C0E466F070E476FE30E41
:10C4A000486FFB0E496F9E0E4A6F070E4B6FFE0ED4
:10C4B0004C6FFB0E4D6FD00E4E6F070E4F6F180E68
:10C4C000506FFC0E516F020E526F080E536F300EFC
:10C4D000546FFC0E556F340E566F080E576F480E92
:10C4E000586FFC0E596F660E5A6F080E5B6F5E0E2A
:10C4F0005C6FFC0E5D6F980E5E6F080E5F6F730EC3
:10C50000606FFC0E616FCA0E626F080E636F870E5C
:10C51000646FFC0E656F666F080E676F9A0E686F2A
:10C52000FC0E696F2E0E6A6F090E6B6FAD0E6C6F8D
:10C53000FC0E6D6F600E6E6F090E6F6FBF0E706F29
:10C54000FC0E716F920E726F090E736FD00E746FC6
:10C55000FC0E756FC40E766F090E776FE00E786F64
:10C56000FC0E796FF60E7A6F090E7B6FF00E7C6F02
:10C57000FC0E7D6F280E7E6F0A0E7F6FFF0E806FA0
:10C58000FC0E816F5A0E826F0A0E836F0D0E846F40
:10C59000FD0E856F8C0E866F0A0E876F1B0E886FDF
:10C5A000FD0E896FBE0E8A6F0A0E8B6F290E8C6F7F
:10C5B000FD0E8D6FF00E8E6F0A0E8F6F360E906F20
:10C5C000FD0E916F220E926F0B0E936F420E946FC1
:10C5D000FD0E956F540E966F0B0E976F4E0E986F63
:10C5E000FD0E996F860E9A6F0B0E9B6F5A0E9C6F05
:10C5F000FD0E9D6FB80E9E6F0B0E9F6F650EA06FA8
:10C60000FD0EA16FEA0EA26F0B0EA36F700EA46F4A
:10C61000FD0EA56F1C0EA66F0C0EA76F7B0EA86FEC
:10C62000FD0EA96F4E0EAA6F0C0EAB6F850EAC6F90
:10C63000FD0EAD6F800EAE6F0C0EAF6F8F0EB06F34
:10C64000FD0EB16FB20EB26F0C0EB36F990EB46FD8
:10C65000FD0EB56FE40EB66F0C0EB76FA20EB86F7D
:10C66000FD0EB96F160EBA6F0D0EBB6FAB0EBC6F21
:10C67000FD0EBD6F480EBE6F0D0EBF6FB40EC06FC6
:10C68000FD0EC16F7A0EC26F0D0EC36FBC0EC46F6C
:10C69000FD0EC56FAC0EC66F0D0EC76FC50EC86F11
:10C6A000FD0EC96FDE0ECA6F0D0ECB6FCD0ECC6FB7
:10C6B000FD0ECD6F100ECE6F0E0ECF6FD40ED06F5D
:10C6C000FD0ED16F420ED26F0E0ED36FDC0ED46F03
:10C6D000FD0ED56F740ED66F0E0ED76FE30ED86FAA
:10C6E000FD0ED96FA60EDA6F0E0EDB6FEB0EDC6F50
:10C6F000FD0EDD6FD80EDE6F0E0EDF6FF20EE06FF7
:10C70000FD0EE16F0A0EE26F0F0EE36FF90EE46F9C
:10C71000FD0EE56F3C0EE66F0F0EE76FFF0EE86F44
:10C72000FD0EE96F6E0EEA6F0F0EEB6F060EEC6FEB
:10C73000FE0EED6FA00EEE6F0F0EEF6F0C0EF06F92
:10C74000FE0EF16F430EF26FF36BF56BF66BF76B4A
:10C75000F86BF96BFA6BFB6BFC6BFD6BFE6BFF6BA5
:10C760000901006B016B026B036B046B07014899B5
:10C770000901056B066B076B086B096B0A6B0B6B8A
:10C780000C6B0D6B0E6B0F6B106B116B126B020E43
:10C79000136F146B010E156F030E166F040E176FD7
:10C7A000050E186F060E196F070E1A6F080E1B6F15
:10C7B000090E1C6F0A0E1D6F1E6B1F6B206B0F0E78
:10C7C000216F000134EF10F0EFEF10F09EEC11F04C
:10C7D00009013E6B090E3D6F030E3F6F000158ECDF
:10C7E00011F001C044F065EF13F054EF18F0A3EF1F
:10C7F00019F033EC25F0CAEC25F0DCEF25F0E6EF7C
:10C8000025F0E9EF25F0EEEF25F005EF26F088EFB3
:10C8100026F0100E486E8651F0090901226F256F2F
:10C82000266B0001A9EC27F0428241A0FED741907F
:10C8300083703DEF29F0C2EF2AF042A208D086C0F3
:10C8400025F9010E0901266F0001A9EC27F0070167
:10C850004751FC0F20E2040F000153EF64F06EEF2C
:10C860002DF0070118D03DEF32F0070114D04850E9
:10C87000F00B100807E075EF46F08751030802E15E
:10C88000CBEF48F052EF56F0070105D04FEF5BF0C9
:10C89000070101D00701472B4751030801E2476B0D
:10C8A0000001C3D70300F2CF21F0F29CF29EE824EE
:10C8B000F76AF736D70FF66EC80EF722000EF86E3D
:10C8C000FB6E0A00F550FA6E0800F55021BCF28CA0
:10C8D00021BEF28EF96E5EC866C86EC88CC8FFFFB6
:10C8E000FFFFFFFFFFFFFFFFFFFFFFFFFFFFFFFF58
:10C8F000FFFFFFFFFFFFFFFFFFFFFFFFFFFFFFFF48
:10C90000FFFFFFFFFFFFFFFFFFFFFFFFFFFFFFFF37
:10C91000FFFFFFFFFFFFFFFFFFFFFFFFFFFFFFFF27
:020000040001F9
:020000040030CA
:0E0000000002161EF3828100FF80FF80FF4089
:020000040020DA
:08000000FFFFFFFFFFFFFFFF00
:00000001FF
